:020000040800F2
:1000000038300020219100080D8E00080F8E000866
:10001000118E0008138E0008158E000800000000E5
:100020000000000000000000000000001D7C00082F
:10003000178E000800000000C57B0008497B0008FF
:100040005191000855910008599100085D910008F0
:100050006191000865910008699100086D910008A0
:10006000719100087591000879910008198E0008B7
:100070007D91000881910008859100088991000810
:100080008D910008919100089591000899910008C0
:100090009D910008A1910008A5910008A991000870
:1000A000AD9100081F8E0008B1910008B5910008BD
:1000B000B9910008BD910008C1910008C5910008E0
:1000C000C9910008CD910008D1910008D591000890
:1000D000D9910008318E0008DD9100086D8E00086E
:1000E000E1910008E5910008E9910008ED91000810
:1000F000F1910008F5910008F9910008FD910008C0
:100100000192000805920008099200080D9200086B
:100110001192000815920008199200081D9200081B
:100120002192000825920008299200082D920008CB
:100130003192000835920008399200083D9200087B
:100140004192000845920008499200084D9200082B
:100150005192000855920008AB8E00085992000891
:100160005D9200086192000865920008699200089B
:100170006D9200087192000875920008000000005E
:10018000799200087D92000881920008859200080B
:10019000899200088D9200089192000895920008BB
:1001A000999200089D920008A192000840F020005A
:1001B00070472DE9F14FB0B0924604910DF1420124
:1001C0003A9A2B9199464A7000200AE01AF8011BCE
:1001D0000498309A90470028049000F034860D98D7
:1001E000401C0D909AF8000050B12528EED1002156
:1001F00000220791089209910A920B910C9204E057
:100200000D9800F022BE41F001011AF8010F2028DC
:10021000F9D023280CD02B2804D02D2805D0302845
:1002200009D00BE041F00201EFE741F00401ECE7F7
:1002300041F00801E9E741F01001E6E72A280FD173
:10024000D9F8002052F8040BC9F8002000280F90BC
:1002500003D540420F9041F004010AF1010A14E075
:100260000F92DFF8EC3B0AE00F98984205DA00EBBA
:10027000800402EB4402303A0F920AF1010A9AF824
:100280000020A2F130000A28EED39AF800002E28B0
:1002900003D04FF0FF320E9229E01AF8010F2A28FE
:1002A00009D1D9F8000050F8042BC9F800000E92CB
:1002B0000AF1010A1BE02D280CBF0AF1010A0020F7
:1002C00000220E92DFF8884B0BE040B90E9AA24252
:1002D00005DA02EB820503EB4503303B0E930AF18E
:1002E000010A9AF80030A3F130020A2AEDD3ADF8E2
:1002F00040100FF660309AF8001000F0CBFE08B105
:100300001AF8010B8DF842009DF84200682805D1CB
:100310009AF8000068280CD1622106E06C2804BF1E
:100320009AF800006C2804D171218DF842100AF16E
:10033000010A12A806901AF801BBBBF125012CD0C6
:100340001C3900F09481091F022940F29081133971
:1003500000F0AB84093900F08A81891E00F04085E5
:10036000491E00F0ED84491E022940F28081091FD8
:1003700000F0E684491F00F0EF80491E00F09584EC
:10038000491E00F0D780C91E0CD0891E00F08D8454
:10039000C91E00F08A8400F02EBD01230793252199
:1003A00000F026BDD9F8000050F8044BC9F8000051
:1003B000002C059440F0AB802B994878002800F081
:1003C000A1804FF0FF340FF6942000F073FE241A42
:1003D00040F0398500F01BBD01236A4602A9304672
:1003E00000F000FE002840F02E85641EF4D1309607
:1003F000079C12AF74B1309E17F8011B0498B047E8
:100400000028049000F01F850D98401C641E0D907C
:10041000F2D130960A9C3021002C8DF800100CDDB2
:10042000309E01236A4602A9304600F0DBFD002819
:1004300040F00985641EF4D13096059F089C74B184
:10044000309E17F8011B0498B0470028049000F074
:10045000FA840D98401C641E0D90F2D130960B9CCE
:100460003021002C8DF800100CDD309E01236A46EF
:1004700002A9304600F0B6FD002840F0E484641E76
:10048000F4D1309605980899099C471874B1309EAC
:1004900017F8011B0498B0470028049000F0D3849B
:1004A0000D98401C641E0D90F2D130960C9C3021AA
:1004B000002C8DF800100CDD309E01236A4602A945
:1004C000304600F08FFD002840F0BD84641EF4D15A
:1004D00030969DF8400041077FF584AE2020002D26
:1004E0008DF800007FF77EAE309C01236A4602A99A
:1004F000204600F077FD002840F0A5846D1EF4D161
:1005000030946FE60FF63C30059000F080BC0E9DF5
:10051000002D04D5204600F0EDFD044607E02A46F4
:10052000204600F0F1FD002814BF041B2C4608945F
:1005300000F06DBCD9F8001051F8040BC9F8001098
:1005400020F00004002121F0FF35CDE9024512AB77
:100550000593782100F040BC2B99487820B14FF0EA
:10056000FF340FF6B02030E79DF84200622860D0DB
:10057000682817D06A283FD06C2806D0712847D049
:1005800074282CD07A281DD062E0D9F8001051F8D8
:10059000040BC9F80010002866D14FF0FF340FF6A5
:1005A0008C2012E7D9F8001051F8040BC9F800109C
:1005B00020B94FF0FF340FF6742006E70D99018043
:1005C00000F025BCD9F8001051F8040BC9F8001050
:1005D000002849D14FF0FF340FF65020F5E6D9F846
:1005E000001051F8040BC9F8001000283CD14FF05E
:1005F000FF340FF63820E8E6D9F8001051F8040B64
:10060000C9F8001080B94FF0FF340FF62020DCE667
:10061000D9F8001051F8040BC9F8001020B94FF0B8
:10062000FF340FF60820D0E60D9AD317C0E9002357
:10063000EDE3D9F8001051F8040BC9F8001020B907
:100640004FF0FF340FF6E410BFE60D990170DEE3C2
:10065000D9F8001051F8040BC9F8001020B94FF078
:10066000FF340FF6C810B0E60D990160CFE39DF896
:1006700042004C2807BFD9F80010CA1DD9F8000065
:10068000C21D22F00702C9F80020D2E90001083299
:10069000C9F80020CDE90201C80F02D007982D212A
:1006A0000AE0BDF84000810702D507982B2103E03E
:1006B000C00705D50798202112AA1154401C0790A5
:1006C00012A807994BF0200300EB010CDDE90201B1
:1006D000CDE92C01612BCDF814C021AC0BD00E98C4
:1006E000002848BF062105D404BF4BF0200067282E
:1006F00001D101210E91DDE902014F0047EAD077D7
:100700007E15FF174FF0FF32974208BF964210D177
:10071000090341EA10510003002908BF002808D04E
:10072000ABF1610503211A2D089118D30FF61C11A6
:1007300010E0DDE902014A00521512F1010F11D15A
:1007400008030FD1ABF1610503211A2D08911FD3C6
:100750000FF600110322604600F002FD57E30FF68A
:10076000E801F7E7DDE902016A4600F005FDCDE9A1
:1007700002014BF02000612811D105983021017051
:10078000821C0592BBF1610F0CBF7821582102E059
:100790000FF6BC01DEE741700798801C0790DDE989
:1007A000020120F0000231F0004308BF002A02D10C
:1007B0000026002542E14BF02008B8F1610F40F01F
:1007C00092800E98002847BF21210191401C019082
:1007D000019FDDE92C017F1C00220023DDE9024599
:1007E00000F002FD38BF85F0004500998DF88420A7
:1007F000091F002F00910DF1850632DD20462946A4
:100800000022002300F00AFD2BD21C2200F020FD64
:1008100004460D4600F0BAFDFF1F002F804609DD9B
:1008200000F0D0FD02460B462046294600F09AFE15
:1008300004460D46F01D0721B8F1000F0CDD491EDE
:100840005EBF08F00F0200F8012D4FEA2818F3D51B
:1008500002E0002200F8012D491EFAD5C61D002F26
:10086000CCDC0DF18500361A01980DF18504864225
:10087000D8BF304600282FD4B04206DA0DF18501EA
:100880000A5C082AA8BF0F2100DA0021024621AB2A
:10089000134400E0401E13F80159521E8D42F9D056
:1008A0000F2904D10DF185018B5C5B1C8B54002A50
:1008B00004D50099091D21AC401C0091411E0BD4A8
:1008C000621813783033DDB23A2DA4BF5B443A3B53
:1008D000491E02F80139F4D50E99002940F1AC8087
:1008E000421E0E92A8E00099DFF8E82647F29750E2
:1008F000414391FBF2F20092DDE92C45C2F107027F
:10090000002A25F0004504DD2046294600F03EFB84
:100910000BE052420020DFF8C01600F037FB024621
:100920000B462046294600F08FFE04460D46B8F1DE
:10093000660F06BF009F0A3706270E983F18142F30
:10094000C8BF142730208DF884000DF18506002FD4
:1009500034DD2046294600F09BFF01460A4606F199
:10096000080304200A26B2FBF6F606EB860EA2EB7D
:100970004E02303203F8012C0A22B6FBF2F202EBEF
:10098000820EA6EB4E063036401E03F8026DE9D10A
:10099000083F002F03F10806D9DD084600F08AFF62
:1009A00002460B462046294600F0DCFD0022DFF817
:1009B0002C3600F08DFF04460D46CAE70DF1850088
:1009C000361A0DF1850404E00098401E761E009052
:1009D000641C20783028F7D0B8F1660F02D1009857
:1009E000401C04E0B8F1650F0CBF012000200E99F7
:1009F00040188642B8BF701E00281DD4B04204DAE9
:100A0000215C3429C8BF392100DC30210246631E35
:100A10009D1800E0401E15F80169521E8E42F9D063
:100A2000392902D1A15C491CA154002A04D500999E
:100A3000491C1C46401C00910646009D0E9F30B28A
:100A4000002802DC01260FF210644BF0200066281B
:100A500008BF6D1C15D067280FFA85F841D118F131
:100A6000040F44DBB84542DA9DF840006D1C0107D5
:100A700003D430B2B842D8BF074628B23F1A48BFA5
:100A800000270FFA85F8B8F1000F00F3AF8008983F
:100A9000411C0891302205990A54002F03DC9DF86F
:100AA0004000010705D50898411C08912E220599A0
:100AB0000A5417EB080FB8BF7D422DB26842ED19FA
:100AC00032B20B909542B8BF2E46059B089836B2BD
:100AD000099632462146184400F042FBAD1B0C95A6
:100AE000CCE0BBF1610F15D14FF0700B17E030B2C5
:100AF000B84204DA9DF840100A0758BF07467F1E27
:100B000048BF0027BBF1670F14BF4FF0450B4FF0F4
:100B1000650B04E0BBF1410F08BF4FF0500B089884
:100B2000411C0891002F059914F8012B0A5403DC8D
:100B30009DF84000010719D50898411C08912E2204
:100B400005990A54002F11DD761E30B28742B8BFD6
:100B50003E460598089B32B22146184400F000FB3F
:100B6000089836B23018BF1B08900B970598089963
:100B70000844B8F1000F80F800B003D42B22427073
:100B8000821C04E02D2145464170821C6D420021EB
:100B90002CAB28460AE004460A2094FBF0F000EB58
:100BA0008005A4EB450403F8014B491C00B2002862
:100BB000F1DC012906DC4BF02000652804BF302061
:100BC00002F8010B00292CAB08D1302002F8010BF0
:100BD00006E0491E585C303002F8010B0029F8DCB1
:100BE000059908980844121A099247E030B229B2D0
:100BF00088421BDA0598089B32B22146184400F05F
:100C0000AFFA089936B271180891A8EB0600002FC8
:100C10000B9003DC9DF84000020705D5059A2E20B5
:100C200050540999491C09910C9727E00598089B95
:100C30002AB22146184400F093FA0898761B4044E3
:100C4000002F089003DC9DF840100A0704D5411CD2
:100C500008912E2205990A5430B28742B8BF3E4609
:100C60000598089B32B204EB0801184400F078FAAA
:100C7000089836B23018BE1B08900B969DF84000BD
:100C800000F01400102840F0C280079A08980B99D1
:100C9000821809988A1882180C980F99801888422F
:100CA00080F2B580081A0A90B1E09DF842006228EF
:100CB00008D068280ED06A2814D06C281FD071285C
:100CC00010D01CE0D9F8001051F8040BC9F800103E
:100CD000C0B21AE0D9F8001051F8040BC9F800109E
:100CE00080B212E0D9F80000C21D22F00702C9F854
:100CF0000020D2E900010832C9F8002006E0D9F846
:100D0000001051F8040BC9F800100021CDE90201D0
:100D10009DF8400001075AD5DDE90223002B08BFEA
:100D2000002A54D04BF02000782850D1079812A9FF
:100D300030220A54401C431C079301F800B046E0DF
:100D40009DF84200622808D068280ED06A2814D086
:100D50006C281FD0712810D01CE0D9F8001051F871
:100D6000040BC9F8001040B21AE0D9F8001051F88D
:100D7000040BC9F8001000B212E0D9F80000C21D3F
:100D800022F00702C9F80020D2E900010832C9F8B0
:100D9000002006E0D9F8001051F8040BC9F8001043
:100DA000C117CDE90201002902D507982D210AE0DB
:100DB000BDF84000810702D507982B2103E0C0074A
:100DC00005D50798202112AA1154401C079012A89B
:100DD000079901440591594602A800F04DF816E024
:100DE00001200790D9F8000050F8041BC9F8000052
:100DF0008DF848100BE001212522BBF1000F07916F
:100E00008DF8482003D0022207928DF849B00F9D3B
:100E100007990A986D1A08992D1A0B986D1A099955
:100E20002D1A0C986D1A9DF840102D1A48073FF5A1
:100E3000DFAA2021002D8DF800107FF7D9AA309E5F
:100E40002C46FFF7C9BA4FF0FF3031B0BDE8F08F44
:100E5000CBCCCC0C686A6C747A4C00007072696EF2
:100E600074665F733A206261642025732061726743
:100E7000756D656E740000002DE9FC4707468A46D3
:100E80003C6950466F2808BF082505D0FFF78EF94A
:100E9000782814BF0A251025D7E900013C26804692
:100EA0008946BAF1640F18BFBAF1690F05D100295C
:100EB00003D5D8F1000869EB4909B9F1000F08BF63
:100EC000B8F1000F0CD1386B50B9082D3AD197F812
:100ED0003800010736D530223B2684F83B2031E02C
:100EE0008DF800A0404649462A46EB1700F0C6FDA3
:100EF0003032D0B2761E3A2801960EDAA25540461C
:100F000049462A46EB1700F0B9FD80465FEA010921
:100F100008BFB8F1000F05D108E09DF800001218D5
:100F2000513AEBE7F868A1198842DBD3082D09D1C3
:100F300097F83800010705D5A05D302802D0761E4D
:100F40003020A055C6F13C03BB61A119F960386B94
:100F5000834208DAC31A3B624FF6EF70398F0140C3
:100F60003987BDE8F38700280ED597F8380000F0E0
:100F70001400102808D17A6B7969386A521A121A4B
:100F8000D21A002AC8BF3A62BDE8F3872DE9D043E0
:100F900006460F4614464FF00008DFF8449012E072
:100FA000E00707D542464B463046394600F090FCF4
:100FB00006460F464046494642464B4600F088FCEE
:100FC000641080468946002CEAD130463946BDE897
:100FD000D0830000A08601000000F03F84D7974135
:100FE00000002440F8B505460E4617461C46002072
:100FF0005CB117F8011BB068A847B06030B1F06A67
:10100000401CF0620020641EF3D1F2BD4FF0FF30AF
:10101000F2BD00007072696E74665F733A20256ECF
:1010200020646973616C6C6F776564007072696EBF
:1010300074663A2062616420256E20617267756D66
:10104000656E7400000000006E616E004E414E003F
:10105000696E6600494E4600300030B5016884680C
:101060004218416802EB5103C90703D54C4401E023
:10107000491C08D19A4218BF12F9011B01D10C304A
:1010800030BD12F8015B002904F8015BF0D4491E61
:10109000F7D5EFE7C9B202788A421AB11CBF10F83F
:1010A000012FF9E718BF002070470268531C036046
:1010B0001170704780B500B906A005490B681BB1D7
:1010C00022220021984701E000F05BFD222002BDB2
:1010D000302C0020636F6E73747261696E742068C7
:1010E000616E646C65723A20626164206D65737331
:1010F0006167650000F1010310F8011B11B110F8E0
:10110000011BFBE7C01A7047C9B2830706D0521E05
:1011100022D310F8013B9942F7D11FE0083A13D3CC
:1011200002F1040241EA012141EA014150F8043B85
:10113000121F21BF4B40A3F1013C2CEA030C1CF011
:10114000803FF3D0C9B2001F083210F8013B521E95
:1011500028BF91EA030FF8D818BF0120401E70473E
:101160004AB1000011F8013B521E00F8013B1CBFC0
:1011700011F8013BF8E7704710B5144600F002F88B
:10118000226010BDC1F30A5343B14A0012F5001F9B
:1011900028D2A3F2FE32A1EB0251704750EA410C73
:1011A00020D001F0004C31EA0C01B1FA81F204BF09
:1011B000B0FA80F3D2180B3AB2F120032CBF00FA38
:1011C00003F1914041EA0C013EBFC2F1200C20FA2C
:1011D0000CF319439040524240F2FD33D21A01EB16
:1011E000035170470022704741EA030C50EA4C0C4F
:1011F00052EA0C0C4FF4001C09D307D01CEB410F32
:101200009CBF1CEB430F8B4208BF824270471CEB14
:10121000430FFBD8994208BF9042704741EA030C44
:1012200050EA4C0C52EA0C0C4FF4001C09D307D0C6
:101230001CEB410F9CBF1CEB430F994208BF90422F
:1012400070471CEB410FFBD88B4208BF82427047AE
:10125000124254D440F2FF7C1CEA11530FD0634574
:1012600031D09B1863453CBF01EB0251704701F040
:10127000004141EA0C510020AFF30080704750EA72
:10128000410320D001F0004C91EA0C011CD0B1FACE
:1012900081F30B3B9A420DD9D21A994051EA0C01C5
:1012A000C3F1200C20FA0CFC61449840531C40F21E
:1012B000FF7CD7E7914041EA0C01C2F1200C20FAF3
:1012C0000CF3194390407047B0FA80F31533202B8C
:1012D000E0D3202AEED3203A203B9A4209D9D21AF1
:1012E00000FA03F141EA0C010020531C40F2FF7C9C
:1012F000B8E700FA02F141EA0C01002070475242BF
:1013000040F2FF7C1CEA11530DD06345DBD0B2EBF9
:10131000030C3CBFA1EB025170470CF1010221EA22
:10132000035141F4801150EA410CCCD001F0004C43
:10133000352A27DC30B481EA0C01B2F1200309DA46
:10134000C2F12003044601FA03F5D0402843D140FE
:101350009C400CE0C3F12002450020FA03F418BFC2
:1013600044F0010421FA03F091400C43002174F190
:10137000004550F1000051EB0C01244230BC7FF4D9
:101380007BAF70476146002076E70000C1F30A5347
:1013900040F21E42D31A0CDDCA0283F3070342EA6D
:1013A000505242F00042DA4002EBE17282EAE17010
:1013B00070476FEAE17203F2E13008B182F0004059
:1013C0007047000010F0004160B148BF4042B0FAE1
:1013D00080F29040D21CC2F5846241EA025202EBD4
:1013E000D02140057047000070B491EA030F4FF020
:1013F000004540F1BF806B40841A71EB030604D2B4
:101400006E40001BB141121973414FF4001C1CEBDC
:10141000410F34BF7CEB430683E00C0DA4EB135665
:10142000362E00F37C80012E45EAC32341DC43EADB
:10143000525312BFD20292025B08240545EAC12131
:1014400041EA5051D2EBC020994125D407D1B0FADE
:1014500080F610FA06F162D00020203608E0B1FADA
:1014600081F6B140C6F1200220FA02F21143B040E9
:101470004FEAF474B4EB465434F001064FEA7404B6
:101480000AD8D6F50016760D04F00044F04061FA53
:1014900006F25040F1404840C00A40EA415021F075
:1014A000004128BF5FEA500550F1000044EBD12114
:1014B00035E0DB0A45EAC121C90AB6F120050EDD97
:1014C00042EA0242120CC5F1200603FA06F6EB408E
:1014D00042EA06056D42984161F100010DE062FAB1
:1014E00006F5F240554063FA06FC82EA0C02F3402E
:1014F0005A406D42904161EB030111F4801F05D108
:10150000641E620502D06D004041494121F4801102
:10151000430875F1004350F1000041EB045170BCE9
:1015200070471CEB410F15D223F0004352EA4306EB
:101530000BD04FEA4C0CBCEB410F04D80C0D661ECF
:10154000342EB7DDEBE7801A994150EA410608BF17
:101550000021E4E708BF1CEB430F28BF6FF0000138
:10156000DDE7000070B491EA030F4FF000457FF50E
:1015700043AF6B40841A71EB030603D2001BB141E9
:10158000121973414FF4001C1CEB410F34BF7CEB6C
:10159000430442E00C0DA4EB1356352E4FDC45EA14
:1015A000C323DB0A45EAC121C912B6F120050DDDCE
:1015B00063FA05F6EB4086EA0305124218BF45F0D0
:1015C0000105C01851F100010CD213E062FA06F5D2
:1015D000F2405540F3415A40B340F3405A4080181E
:1015E000594107D349085FEA30005FEA350528BF53
:1015F00045F0010501F58011420875F1004250F1F6
:10160000000041EB04514E0016F5001F70BC38BFBE
:1016100070470020090D090570471CEB410F10D2DF
:1016200052EA43060BD0BCEB410F05D80C0DAB437F
:10163000661E342EB6DD02E0AB438018594170BC03
:10164000704770BC70470000F0B540F2FF7581EA4A
:10165000030C0CF0004C15EA11541DBF15EA13578A
:10166000AC42AF42E5E0BC41C1F31301C3F3130345
:10167000801A994143F4801304D2641E0018494132
:1016800080185941C90241EA5051B1FBF3F603FBFE
:101690001611A2FB0675D7EBC020A94102D2761E17
:1016A00080185941C90241EA5051B1FBF3FE03FBD6
:1016B0001E11A2FB0E75D7EBC020A94103D2AEF1DB
:1016C000010E80185941890241EA9051760546EA97
:1016D0008E2EB1FBF3F603FB1611A2FB0675D7EBBA
:1016E0008020A94102D2761E80185941C90241EAE0
:1016F00050514EEA060EB1FBF3F603FB1611A2FBA6
:101700000675D7EBC020A94102D2761E8018594138
:10171000C90241EA5051B1FBF3F703FB1711A2FBD9
:101720000735D3EBC020A94167F100070CBF004289
:1017300047F0010766F3D5274FEA1E31B80814F5C4
:10174000806412DDBD0775F1004250EB0E5051EB85
:10175000045111F5801F5CBF41EA0C01F0BD4CF053
:101760007F6141F0E0410020F0BDBD076D0840EA17
:101770000E5041F48011D4F10104B4F120060ADACC
:10178000C4F120060200E04001FA06F3E1401843EC
:10179000B24015430EE0342C13DCC6F1200445EAB8
:1017A00040056D0820FA06F2154321FA06F0A14023
:1017B0000D43002175F1004250F1000051EB0C0186
:1017C000F0BD00205FEA0C01F0BDCFB992185B417B
:1017D000B3FA83F704BFB2FA82F6BF190B3FB7F131
:1017E00020062FBF02FA06F3BB40C7F1200622FAFB
:1017F00006F638BF3343BA401CB1E419641E33E720
:101800007F4231F00041B1FA81F404BFB0FA80F6B2
:10181000A4190B3CB4F120062FBF00FA06F1A14039
:10182000C4F1200620FA06F638BF3143A0403C1B25
:101830001AE7AC421ABF05EA1357AF4212E050EA6A
:1018400041061CBF52EA4306BFE750EA4107304653
:1018500061461CBF41EA0551F0BD52EA430C08BF86
:10186000C143F0BD00204FF4001616EB410F98BFA6
:1018700016EB430F08BF16EB410F24BFC14305E031
:1018800016EB430F0CBF61464CEA0551F0BD00005A
:10189000400D40F21E4C40EAC120BCEB115C40F010
:1018A000004003D48CF30701C84070476FEAE17031
:1018B0007047000050B1B0FA80F18840C91CC1F5F2
:1018C0008461090501EBD02140057047014670474E
:1018D00030B540F2FF7C1CEA11541DBF1CEA1355C1
:1018E000644565453FE0641981EA030C6FF35F537B
:1018F0000CF0004C43F48013C90241F0004141EA6E
:10190000505EC5021100A5FB020200284FF0000046
:10191000EEFB01204FF00001E3FB052118BF42F070
:101920000102401800214941E3FB0E01A4F5806447
:101930000D0302D292184041494154F1010470DD77
:10194000450872F1004250F1000051EB0451A1F53D
:10195000801102D441EA0C0130BD40F2FF7E4CEA16
:101960000E51002030BD0CEA1355644518BF654583
:1019700081EA030C0CF0004C41D050EA410E1CBF30
:1019800052EA430E02E06146002030BD24422C445E
:101990001BD15FEA050EF6D0090302BF0146002005
:1019A000AEF1140EB1FA81F5AEEB050401FA05FEB5
:1019B0000C35C5F1200100FA05F5C8404EEA000ECD
:1019C0006FF35F5343F480139CE733F00043B3FAA3
:1019D00083F504BFB2FA82FE75440B3D641BB5F17A
:1019E000200E2FBF02FA0EF3AB40C5F1200E22FAF3
:1019F0000EFE38BF43EA0E03AA40641C7CE750EA9F
:101A0000410E14BF52EA430E6FF000014FF400156F
:101A100015EB430F8EBF194615EB410F9DE7B4D868
:101A200030BDD4F10104B4F120050FDAC4F1200572
:101A3000520828BF42F0010210FA05FE01FA05F52E
:101A40007244E2BFE0402843E1400FE0352C9ADCCD
:101A5000C5F1200452EA400220FA05F218BF42F014
:101A6000010231FA05F0A1400A43002172F100425F
:101A700050F1000051EB0C0130BD0000D3BBD9B1D7
:101A8000B2F5803F5BD2022A1ED98C46B1FBF2F13F
:101A900002FB11C31B0443EA1043B3FBF2FC02FB3D
:101AA0001C3380B240EA0343B3FBF2F002FB103276
:101AB00040EA0C4000237047022A05D98446B0FB57
:101AC000F2F002FB10C270474AB105D100F00102EA
:101AD00049085FEA3000704700220023704700F099
:101AE00053B80B000200002100207047F7D30022FA
:101AF00000237047904271EB030CF2D370B5B1FA3A
:101B000081F4B3FA83F52C1BA340C4F1200532FA0B
:101B100005F63343A2405FF00046E64002E05B0872
:101B20005FEA3202841A71EB030524BF204629467E
:101B30007641F4D302000B003000002170BD70B577
:101B4000B1FA81F4B2FA82F5C4F120046419B4F157
:101B50002006DAD3B2405FF00044F440002502E0F2
:101B600052085FEA3303C61A71EB020E24BF3046F7
:101B7000714664416D41F3D302000B00200029003F
:101B800070BD012000F002B87047000080B5AFF3CF
:101B90000080024A11001820ABBEFBE726000200BD
:101BA00038B5040001D1012032BD00F04DF918B95B
:101BB00000F085FB00F0D9FE85E090F83D1001298A
:101BC00001D001207047022180F83D10DFF82C225F
:101BD0000168914218BFB1F1804F12D0DFF8202286
:101BE00091421CBFDFF81C3299420AD0DFF818225C
:101BF00091421FBFDFF814329942DFF8142291425C
:101C000009D18B68DFF818121940062918BFB1F501
:101C1000803F05D001680A68084642F00102026070
:101C20000020704701680A6A41F211131A4202BF8C
:101C3000096A40F24442114239E090F83D1001290E
:101C400001D001207047022180F83D100168CA6868
:101C500042F00102CA600168DFF8A021914218BF7A
:101C6000B1F1804F12D0DFF8982191421CBFDFF80C
:101C7000943199420AD0DFF8902191421FBFDFF8DA
:101C80008C319942DFF88821914209D18B68DFF8C5
:101C900090111940062918BFB1F5803F05D00168A1
:101CA0000A68084642F0010202600020704705D130
:101CB00001680A6852080B4652001A60012180F838
:101CC0003D100020704702206870211D206800F040
:101CD000FAFA012028730121A970E870297168714E
:101CE000A971E87129726872A972E872697000209E
:101CF00032BD38B5040001D1012032BD00F0A4F896
:101D000018B900F0DCFA00F0ABFEDCE770B5044671
:101D100004F13E0009B902780FE0042908BF4278B7
:101D20000BD0082908BF827807D00C2908BFC278D9
:101D300003D010290CBF02794279012A01D0012079
:101D400070BD11B90222027014E0042902D10222EE
:101D500042700FE0082902D1022282700AE00C29A9
:101D600002D10222C27005E0102907BF02220271CF
:101D7000022343712068012200F0C3FC00F038F810
:101D800018BF904208D088421FBFDFF89850A84281
:101D9000DFF89460B04203D1456C45F400454564DA
:101DA0002068984218BFB0F1804F0BD000F018F8AF
:101DB0001CBF144DA84205D000F00FF81CBF904284
:101DC000884206D100F00FF818BFB0F5803F02D06E
:101DD000206800F01FF8002070BD0B4B9842704740
:101DE000074B9842704781680D48084006287047A5
:101DF0002068024B0649054A98427047002C014072
:101E00000004004000080040000C00400034014085
:101E1000004001400168024641F001011160704735
:101E200007000100004401400048014038B50400AB
:101E300001D1012032BD00F007F818B900F03FFAD7
:101E400000F069FDFFF73FBF04F13C05687870477B
:101E500070B504000E4601D1012070BDFFF7F4FFFC
:101E600018B900F02CFA00F0FCFD02206870211D6A
:101E7000206800F028FA2068016821F0080101605C
:101E80000121206802681643066001202873A970AA
:101E9000E870297268726970002070BD70B50446E0
:101EA0002068C5680669B10714D5AA0712D56FF076
:101EB0000201016101222277806910F0030F2046A0
:101EC00002D000F0CFFD03E000F0CDFD00F086F879
:101ED00000202077700715D5690713D520686FF0AB
:101EE0000402026102212177806910F4407F2046BC
:101EF00002D000F0B7FD03E000F0B5FD00F06EF891
:101F000000202077300715D5290713D520686FF0FA
:101F10000802026104212177C06910F0030F2046F6
:101F200002D000F09FFD03E000F09DFD00F056F8A8
:101F300000202077F00615D5E90613D520686FF04C
:101F40001002026108212177C06910F4407F204609
:101F500002D000F087FD03E000F085FD00F03EF8C0
:101F60000020207706F0010105F00100014206D0B3
:101F700020686FF001010161204600F0EAFD3006A3
:101F800008D5290606D522686FF08000106120462A
:101F900000F018FEF00508D5290606D522686FF472
:101FA00080701061204600F00EFE700608D56906AC
:101FB00006D522686FF040001061204600F004FE54
:101FC000B0060AD5A90608D522686FF02000106176
:101FD0002046BDE8704000F0F8BD70BD204600F01E
:101FE000F5BDF8B500F005F901D10220F2BD0120E0
:101FF00084F83C007AB9F36872683168206800F0B0
:10200000F1FA2168886920F00C0088618A69B0685B
:1020100002438A6163E0042A10D1F3687268316870
:10202000206800F034FB2068816921F440618161FF
:102030008169B26841EA0221816150E0082A24D115
:102040002168F068726833681C311B024F68D1F850
:1020500004C02CF4807CC1F804C027F42067D1F8B8
:1020600000C04FEA9C0C42EA8C0260F3071203F4B2
:1020700020630A603B434B60086820F00C00086056
:102080000A68B06802430A6029E00C2A26D1206859
:10209000F168726833681C301B034768D0F804C0CD
:1020A0002CF4805CC0F804C027F42047D0F800C0AE
:1020B0002CF4407C4CEA022C61F30F3C03F42043E7
:1020C000C0F800C03B434360016821F440610160F7
:1020D0000268B16842EA0122026000E0012500F0D6
:1020E00001F8F2BD002084F83C002846704770B526
:1020F00000F07FF801D1022070BD012084F83C007F
:1021000052B1042A19D0082A29D00C2A38D0102A12
:1021100048D0142A57D068E0206800F02FF92168D1
:10212000886940F008008861886920F004008861AF
:102130008A69306902438A6158E0206800F060F9DA
:102140002068816941F400618161816921F48061C5
:1021500081618169326941EA0221816146E020683A
:1021600000F086F92168C86940F00800C861C869B4
:1021700020F00400C861CA6930690243CA6135E0D1
:10218000206800F0B0F92068C16941F40061C161C4
:10219000C16921F48061C161C169326941EA0221EA
:1021A000C16123E0206800F0C5F92168486D40F066
:1021B00008004865486D20F0040048654A6D3069A4
:1021C00002434A6512E0206800F0DEF92068416DA4
:1021D00041F400614165416D21F480614165416DCB
:1021E000326941EA0221416500E00125FFF77AFFEB
:1021F00070BD0446002594F83C0001280E46704747
:1022000070B5064606F13C0500242878012801D166
:10221000022070BD0120287002226A70DFF81C04C1
:1022200032689368034093600868020018BF102862
:1022300030D0202818BF30282CD0402826D0502855
:1022400019D060281BD0702806D0B0F5805F27D049
:10225000B0F5005F07D022E000F02CF8306881680C
:1022600041F0770105E000F025F83068816841F41D
:102270008041816014E000F019F850210BE0CA6839
:102280004968306800F019FA602104E000F00EF8A7
:10229000402100E00146306800F021FA00E001240E
:1022A0000120687000F00BF870BD0000CA68496832
:1022B0003068DDE1CB684A688968306817E2002140
:1022C0002970204670472DE9F043D0F800C0DFF8B0
:1022D0007073DFF87033DFF87043DFF87053DFF8A6
:1022E0007063DFF87023DFF870E3DFF87083B842C3
:1022F00018BFB0F1804F07D0404518BF704503D0DC
:10230000904218BFB0420FD12CF07009D1F804C030
:102310004CEA090CB84218BFB0F1804F0CD04045D0
:102320001CBF7045904207D0B04218BFA84203D0EE
:10233000A04218BF984205D12CF44072D1F80CC0CD
:102340004CEA020C4A692CF0800C42EA0C0CC0F8F2
:1023500000C0B842D1F808C0C0F82CC00A68826238
:1023600018BFB04204D0A8421CBFA042984201D17D
:102370000969016301224261BDE8F0832DE9F04162
:10238000066A026ADFF8B882DFF8BC72DFF8BCC206
:10239000DFF8BCE252085200026226F002064368EF
:1023A0008569DFF8BC220C6815402C438D683543E5
:1023B000DFF89062404518BF704504D060451CBFEF
:1023C000B842B0420DD1CA6825F00805154325F082
:1023D0000405404518BF704505D0604518BFB84298
:1023E00001D0B04205D14A6923F440731A438B6986
:1023F000134343608461496841630562BDE8F0812D
:10240000F0B5036A026A974D22F01002026223F0CF
:102410002003446882690E6815408A6845EA0625EB
:1024200043EA021300F05BF818BF904208D1CF686E
:1024300023F0800343EA0713B04223F040030AD09D
:1024400090421CBF814A904205D07F4EB0421CBFD3
:102450007C4A904206D14E698A6924F4406416434E
:1024600044EA860444608561496881630362F0BD83
:10247000F0B5036A026A22F48072026223F40073E8
:102480004468C669764A0D6816408A68354343EA4F
:10249000022300F024F818BF904208D1CF6823F43B
:1024A000006343EA0723B04223F480630AD09042DA
:1024B0001CBF664A904205D0634EB0421CBF614AC1
:1024C000904206D14E698A6924F44054164344EA86
:1024D00006144460C5614968C1630362F0BD584E8B
:1024E0005B4AB042704770B5026A036A5D4C23F4E0
:1024F0008053036222F400524368C56900F06BF810
:1025000042EA0532B0421CBF514DA84207D04F4E9F
:10251000B0421FBF4C4DA8424A4EB04204D14D6953
:1025200023F4804343EA85134360C461496801642E
:10253000026270BD70B5036A026A414E22F48032B5
:10254000026223F400334468456D474A15400A6827
:102550002A438D6843EA0543B0421CBF3C4DA84264
:1025600007D03A4EB0421FBF374DA842354EB04259
:1025700004D14D6924F4803444EA05244460426562
:1025800049688165036270BD70B5026A036A374CA1
:1025900023F48013036222F400124368456D00F0B7
:1025A0001AF842EA0552B0421CBF294DA84207D092
:1025B000264EB0421FBF244DA842224EB04204D145
:1025C0004D6923F4802343EA8523436044654968C9
:1025D000C165026270BD0E682C4044EA06248D6815
:1025E000174E7047F0B5046A056A154E6D086D0008
:1025F0000562B042856918BFB0F1804F0DD0174E0B
:10260000B0421CBF144FB84207D0124EB0421FBF99
:102610000F4FB8420D4EB04203D1AD0842EA8502D9
:1026200001E045F0010263F3071224F00A0401F00F
:102630000A01826121430162F0BD00008800FEFFB3
:10264000002C01400048014000440140004001408E
:1026500000340140000C004000080040000400402D
:102660008CFFFEFFFF8CFFFE8FFFFEFFFF8FFFFE44
:1026700010B5036A046A64086400046223F00A0364
:10268000846924F0F00444EA0214846144E030B523
:10269000046A056A25F0100505620901856925F4BB
:1026A000407545EA022563F30F3524F0A00401F0DC
:1026B000A00185612143016230BD10B5036A046A3F
:1026C00024F01004046223F0A003846924F470440D
:1026D00044EA0234846143EA0113036210BD826854
:1026E00022F07002114341F007018160704710B57C
:1026F000846824F47F442143114341EA032181602B
:1027000010BD10B501F01F01036A01248C40A343E2
:10271000036202FA01F1036A1943016210BD00006D
:1027200018B587B004A800F047F86846002480E890
:102730001E00DFF800434FF0FF304FF08041E060B3
:1027400021606260A2602261A2612046FFF76EFBF9
:1027500008B100F009FA002104910691204604A96D
:1027600000F036FA08B100F0FFF9002101220091D3
:10277000019202910391042269462046FFF731FC41
:1027800008B100F0F1F908B010BD1FB500F013F862
:10279000A94CAA4921606260A2601F21802200F03A
:1027A00029F808B100F0E0F92021009100220292FE
:1027B0006946204618E0684600210022002380E890
:1027C0000E0070471FB5FFF7F6FF9D4C9D49216035
:1027D0004F2060604FF6FF71A26000F00BF808B167
:1027E00000F0C2F900F07BF800F0F2F908B100F057
:1027F000BBF91FBDE160A2612046FFF7D1B918B552
:1028000099B00AA8002100220023002480E81E00BD
:1028100068468D4C80E80E001C2103A800F064FA85
:102820002C210EA800F060FA88482060002140F2B8
:102830008F10E0606160A1602161022060618021F1
:10284000A1612046FFF7ACF908B100F08DF94FF413
:1028500080500A900AA92046FFF7D2FC08B100F088
:1028600083F92046FFF745FA08B100F07DF9082109
:102870002046FFF7EDFA08B100F076F900F02FF8E6
:1028800000F0A6F908B100F06FF902220592C72105
:102890000491042207926020002103900691089180
:1028A0000022099203A92046FFF721FC08B100F09D
:1028B0005BF900204FF400510E900F901090119092
:1028C0001290139118900EA9204600F0BFF908B19C
:1028D00000F04AF9204600F086F81AB010BD002139
:1028E0000091029120466946704780B55848594981
:1028F00001604F2200234FF6FF7142608360C16088
:10290000036143618361FFF74BF918B1BDE80140F2
:1029100000F02AB901BD10B586B000F086F8226833
:10292000B2F1804F1FD14C48C16841F00101C16034
:10293000C16801F0010100910099026842F00102B2
:1029400002600221006800F00100009000980191EF
:1029500002914FF0904000210391049101210591D3
:1029600001A900F0C5F906B010BD80B50068334A72
:102970003A49904207D1086840F0100008600968A1
:1029800001F0100109E02F4A904208D1086840F098
:1029900020000860096801F0200100910AE02B4A3C
:1029A000904209D1886840F480308860886800F4DB
:1029B00080300090009801BD264A904212D188686C
:1029C00040F4003088600022886800F400300090F5
:1029D0000F210098192000F0ADFABDE8024019203F
:1029E00000F0C6BA01BD10B586B000F01EF822682E
:1029F00016498A4217D11848026842F00102026063
:102A00000421006800F0010000900222009801916A
:102A100002920021039104914FF090400E21059104
:102A200001A900F065F906B010BD0446142101A803
:102A300000F05AB9BC290020082A002000100040EC
:102A4000542A002000140040A02A00200040014029
:102A5000EC2A0020004401404C1002405810024073
:102A6000704770477047704780B500F097FA00F0E4
:102A700039F800F0A9FA00F033FB00F049FB00F050
:102A8000F9FB00F010FC00F028FC00F03BFCFFF725
:102A900047FEFFF77AFEFFF795FEFFF7B0FEFFF760
:102AA00024FF00F063FD00F02FFE00F075FD00F044
:102AB00018FF00F01CFF00BF2CA000F0FCFE00BFC0
:102AC0000FF2F4020FF2E40130A000F0F4FE7F21D7
:102AD000234800F021FF00F0F0FF01F01DF901F0A4
:102AE00067F9FEE780B596B0442105A800F0FCF830
:102AF0001421684600F0F8F84FF4007001F09CF9DA
:102B000008B100F031F84FF4803106910120032123
:102B1000109105900222119014210F92129113929C
:102B20001492159205A801F0BFF908B100F01CF845
:102B30000F2003210090019100220292039204923F
:102B40000421684601F0FDFB08B100F00DF817B054
:102B500000BD00680349884208BF01F05DBD7047B1
:102B600030270020002C014072B6FEE74D696372E9
:102B70006F20436C696D6174652053746174696F73
:102B80006E2053656E736F722E0D0A005665727358
:102B9000696F6E20312E302E30204275696C643A98
:102BA0002025732025730D0A000000004A756C2053
:102BB000203620323032340031313A31323A303737
:102BC0000000000070477047704770477047000072
:102BD000F0B500F13C031A78012A01D10220F0BDC2
:102BE00001221A7002245C700568DFF85CC06E6810
:102BF000AC683A4F654518BFBD4203D126F4700258
:102C00004E6816430A6826F0700616436E60026826
:102C1000624518BFB2F1804F0CD02E4882421CBFD3
:102C20002F4DAA4206D02A4882421EBFBA422D4DDD
:102C3000AA4204D1886824F08004044394600121EE
:102C4000597000201870F0BD002C014030B590F88C
:102C50003C20012A01D1022030BD012280F83C2015
:102C6000CC688A684B681C4D24F44074144324F4E7
:102C700080641C430A680B6924F40064144324F440
:102C800080541C434A698B6A24F40054144324F48E
:102C9000804423438A69046823F4702343EA02438F
:102CA000AC421CBF0D4A94420CD14A6A23F4700313
:102CB00043EA0253CA6923F08073134323F000757B
:102CC0000B6A2B436364002180F83C10002030BD68
:102CD000000C004000040040002C01400034014082
:102CE0000008004000400140002201F09DBC0000AF
:102CF0002DE9F84F0027784A784B4FF00F0805462A
:102D00000E4636E0764CA54214BF082407248C40BA
:102D1000744944EA0E0441F82C40C143D2F808C07B
:102D2000746801EA0C0CE40248BF40EA0C0CC2F8DB
:102D300008C0D2F80CC0746801EA0C0CA40248BFA9
:102D400040EA0C0CC2F80CC0D2F804C0746801EA66
:102D50000C0CA40348BF40EA0C0CC2F804C0D2F823
:102D600000C0746801EA0C01E40348BF014311602C
:102D70007F1C316831FA07F000F09E800124BC40CE
:102D800014EA0100F4D04FEA470C032101FA0CF1D8
:102D90006FEA010E716801F00309B9F1010F1CBF60
:102DA00001F00301022912D1A968D6F80C900EEAAD
:102DB000010109FA0CF949EA0101A960696821EAEF
:102DC00004047168C1F30011B9400C436C60B90090
:102DD000347904F00304032C21D0EC68D6F8089071
:102DE0000EEA040409FA0CF949EA0404EC603479A7
:102DF00004F00304022C12D1FC0805EB840401F05A
:102E00001C09D4F820A008FA09FB2AEA0B0AD6F814
:102E100010B00BFA09F949EA0A09C4F820902C68A5
:102E20000EEA040E347904F0030404FA0CF444EAC4
:102E30000E0CC5F800C0746814F4403F98D0D3F865
:102E400000C0284C4CF0010CC3F800C04FEA970CAE
:102E5000D3F800E00EF0010ECDF800E001F00C0117
:102E6000DDF800E054F82CE008FA01F42EEA040E34
:102E7000B5F1904F08BF00241DD01B4CA54208BFE0
:102E8000012418D0194CA54208BF022413D0184CB5
:102E9000A54208BF03240ED0164CA54208BF042447
:102EA00009D0154CA54208BF052404D0134CA542F7
:102EB0007FF428AF06242AE7BDE8F18F0AB18161CB
:102EC000704781627047426901EA0203914341EA17
:102ED000034181617047000000040140601002401E
:102EE000001C004808000140000400480008004899
:102EF000000C00480010004800140048001800486A
:102F00000901020002D42048815470471F4B02F08F
:102F10000F021A4402F8041C70471D4B19684FF643
:102F2000FF020002114000F4E06008431949084321
:102F30001860704770B5164B1C68C4F30223012457
:102F4000C3F10705052D2EBF0F2504FA05F56D1EEB
:102F50001E1D072E34BF0023DB1E2940994004FAB2
:102F600003F3BDE870405B1E1A401143C8E7000040
:102F7000010007D4012200F01F01074B8A404009DD
:102F800043F820207047000000E400E018ED00E066
:102F90000CED00E00000FA0500E100E0094810B582
:102FA000016841F4807101600320FFF7B6FF0F2034
:102FB00001F054FB0024002814BF012401F096FB0B
:102FC000204610BD0020024070B586B014220021BA
:102FD000684601F0A9FB3A483A4C01683A4D41F085
:102FE0000401016041F60806026802F0040205923D
:102FF0000599026842F080020260036803F08003D2
:1030000005930599026842F001020260036803F02B
:10301000010305930599026842F002020260036809
:1030200003F0020305930599026842F0080202606A
:103030000022006800F0080005904EF2C0310598AB
:103040002046FFF73BFF002231464FF09040FFF74C
:1030500035FF00222C212846FFF730FF4EF2C01129
:1030600000F034F82046FFF743FE012101910222CF
:10307000002103910292009669464FF09040FFF7BD
:1030800037FE2C2100F022F82846FFF731FE4FF4DE
:103090000071009101220021029103910192694681
:1030A0002046FFF725FE4FF440700021009001916B
:1030B000029128466946FFF71BFE06B070BD00006E
:1030C0004C10024000080048000400480091012212
:1030D000019202210291002203926946704700008A
:1030E00080B50A48016841F00101016000220068D2
:1030F00000F001000090052100980B20FFF71AFF57
:10310000BDE802400B20FFF733BF00BF481002406C
:1031100018B589B00C22002106A801F005FB182281
:103120000021684601F000FB4B4C4C482060002118
:10313000042060616160002084F82000E16021616A
:1031400021834FF480600121E062E16104F13000ED
:1031500000224FF4E861A260A16202704260027234
:10316000204601F015FB08B1FFF7FEFC0020069099
:1031700006A9204600F01AFC08B1FFF7F5FC384913
:10318000009106220192022102917F2203920421E2
:103190000491002205926946204601F053FC08B1D3
:1031A000FFF7E2FC0AB010BD30B5A9B00446142206
:1031B000002101A801F0B8FA8C22002106A801F034
:1031C000B3FA20682549884244D14FF480424FF039
:1031D00040510692259106A801F0E4FE08B1FFF7E0
:1031E000C3FC2048204D016841F400510160026891
:1031F00002F4005200920099026842F00402026058
:103200000121006800F00400009003220098174894
:10321000019102920021039101A9FFF769FD0021AC
:103220006960E960802129614FF48061104828605D
:10323000A9614FF48070002268614FF44051AA6088
:10324000EA612962284602F05FF908B1FFF78CFCB9
:103250002565AC6229B030BD302700200000045045
:10326000020030044C100240382B002000080048B7
:103270000800024080B5B048B049B14A01604260E0
:103280000021C1604FF080530C2141618360002216
:1032900000210261826101624262002302F08FFA22
:1032A00000B116E001BD80B5A648A74901604FF402
:1032B000E13200230C2142608360C36003614161FD
:1032C0008361C3610362436202F0C0FA00B100E0AF
:1032D00001BDBDE80140FFF747BC10B59B4C9C48C1
:1032E00020604FF416510C20002260616160A260E2
:1032F000E2602261A261E26122626262204602F023
:10330000A5FA15E010B5934C934820604FF4165180
:1033100061600C20002200216061A260E2602161F6
:10332000A161E161216261620023204602F047FA57
:1033300008B1FFF719FC04F188012046BDE81040F0
:10334000012202F017BB30B5A9B0044614220021B7
:10335000684601F0E9F98C22002106A801F0E4F9A1
:10336000206876497D4C884222D120224FF480612A
:103370000692199100F0C2F808B1FFF7F5FB206939
:1033800040F001002061206900F0010005900598DF
:10339000216841F00201216040F60241226802F0FA
:1033A00002020592022205986D4800F0AAF838E062
:1033B00065496C4D884237D1102200210692189140
:1033C00000F09CF808B1FFF7CFFBE06840F48010F4
:1033D000E060E06800F48010059000F082F8226858
:1033E00002F0040205920598216841F0080121606D
:1033F0004FF48051226802F00802059202220598DB
:1034000000F07FF82846FFF773FC022101910022AB
:10341000042002920321009003910822049269463D
:103420005148FFF765FC5AE0494988421ED1012204
:103430000692149200F062F808B1FFF795FB6069FC
:1034400040F480406061606900F4804000F04FF813
:103450004FF4C061226802F0010200F05CF8002223
:1034600005212520FFF766FD252036E03A498842F0
:1034700035D1042210210692169100F03FF808B1D0
:10348000FFF772FBE06840F48020E060E06800F441
:10349000802000F02CF8226802F00102059200F072
:1034A00020F84FF40041226802F0040200F033F8E3
:1034B00002210191002202924FF44060032100900A
:1034C00003910722049269462846FFF711FC002267
:1034D00005212720FFF72EFD2720FFF749FD29B002
:1034E00030BD0598216841F00401216070470590C6
:1034F0000598216841F001012160704706A801F09C
:1035000051BD0091019200210291032208210491F2
:103510000392694670470592022205980091019234
:1035200000210291032207210491039269464FF082
:103530009040FFF7DDBB0000202600200080004007
:1035400024330300A8260020005000400825002056
:103550000038014094250020004800404C100240F3
:103560000004004800080048000C004810B55F4CFB
:103570005F4800F027F808B1FFF7F6FA002120466F
:1035800002F0F2FE08B1FFF7EFFA0021204602F048
:1035900000FF00B125E010BD10B5564C564800F0B4
:1035A00011F808B1FFF7E0FA0021204602F0DCFE36
:1035B00008B1FFF7D9FA0021204602F0EAFE00B177
:1035C0000FE010BD4D49206000220120E0606160E5
:1035D000A26022616261A261E2612262204602F081
:1035E00003BFBDE81040FFF7BFBA30B5A9B004462D
:1035F00014220021684601F097F88C22002106A8C9
:1036000001F092F820683A493D4C3E4D884221D164
:1036100040224FF4805106921A9106A801F0C2FC94
:1036200008B1FFF7A1FA286840F0020028601222D2
:10363000296801F002010591C02100F04BF82046F5
:10364000FFF756FBE86840F40010E860E86800F413
:1036500000103BE0284988423AD14FF480720021A3
:1036600006921C9106A801F09DFC08B1FFF77CFAB8
:10367000286840F001002860296801F001010591E7
:103680000598296841F00201296080212A6802F02A
:1036900002020592122200F01DF84FF09040FFF751
:1036A00027FB122101910022029210200321009099
:1036B00003910422049269462046FFF719FBE8684B
:1036C00040F40000E860E86800F400000090009812
:1036D00029B030BD0598009101920021029103228A
:1036E000042104910392694670470000C828002015
:1036F000005400401C290020005C0040EC9C90100D
:10370000000400484C10024080B528482849016058
:103710004FF482724FF44071C16042600721C16270
:1037200000234FF48022082183600361436182619A
:10373000C3610362436283620363416303F034F94C
:1037400018B1BDE80140FFF70FBA01BD10B586B052
:1037500004461422002101A800F0E6FF2168144865
:10376000814221D11348C16841F48041C160C168E0
:1037700001F4804100910099026842F00202026067
:103780004FF47041006800F002000090022200989F
:10379000094801910292002103910322052105911C
:1037A000049201A9FFF7A4FA06B010BD002800207A
:1037B000003800404C1002400004004870B5514EE3
:1037C000737804460025A34212D1705D70B9701958
:1037D000083003F059F9012C02D1FFF77EFD03E018
:1037E000032C08BFFFF78EFD01207055701970BDC6
:1037F000707E1825A042E8D0002070BD02B50028D8
:103800001CBF0178002912D04078012804D10A2376
:10381000012269463C4805E0032808D10A23012219
:1038200069463A4802F056F808B9012002BD002066
:1038300002BD38B504460D4606E00D2100F01BF828
:103840000A2100F018F86D1C287830B10A28F4D04D
:1038500015F8011B00F00FF8F6E731BDF8B5044686
:103860000D461646002703E0E95D00F004F87F1CD2
:10387000B742F9DBF1BD2046C0E700281CBF017844
:1038800000291EBF01694069814201D001207047B3
:10389000002070471CB500218DF800100446FFF78A
:1038A000ECFF20B1694604F1080003F00CF9FFE7D2
:1038B0009DF8000016BD0EB478B5154D044605F10F
:1038C000CC0664213046FFF70FFA05AA21463046A0
:1038D00003F012F928683146FFF7ABFF71BC5DF8C1
:1038E00010FB10B50A4CC822211D012005E010B5BF
:1038F000084C4FF49672211D0320FFF75FFF2060F4
:1039000010BD0000C00000200825002094250020E4
:10391000F01F0020202100207CB50446002004F187
:1039200054060D4600903178012901D1022076BD60
:103930000120307000F035F8010070682AD120F4C1
:10394000885040F00200706005F080452268DFF882
:103950005800936803401D4345F00045956020687A
:103960008068C00F10D00098401C00900098B0F5FF
:10397000912FF4D3706820F0020040F010007060C6
:1039800000203070012076BD7268012060F30102D2
:10399000726002E040F01000706000203070084655
:1039A00076BD204601F064BAC0FFFF3F2DE9F0412B
:1039B00000F154049AB023780022012B08BF0220A2
:1039C00052D001252570002616960025179503680C
:1039D000294DAB422CD1294FDFF8A4E03B68DEF83B
:1039E00000506D073AD45B0738D40B68254DDFF8DB
:1039F00098C0264E0BB3D6F800804B6890F8300084
:103A000028F4604843EA080343EA4038C6F80080D7
:103A1000DEF800003B68DCF8007018433843C30749
:103A20001FD43768086889683D4005430D4313E09B
:103A300000F01DF82270012016E0306820F460408C
:103A40003060DEF800003968DCF8003008431843C5
:103A5000C00706D431680D40356002E000F007F879
:103A600001220020207010461AB0BDE8F081606885
:103A700040F02000606070470000045008010450CE
:103A800008000450E0F0FFFF08020450080304504F
:103A900010B50023DAB2825C5140C9B208224C0052
:103AA00009064CBF84F031012146521EF7D15B1C40
:103AB000DAB2022AEEDBC8B210BD1FB50122202106
:103AC00089488A4CFFF7FAF9012003F02FF802A980
:103AD00003A800F083F850B95C21204603F03AF8BF
:103AE000411C512204F13000FFF7E5FE0DE0029881
:103AF00003F03EF8CDE90001039803F039F80246DF
:103B00000B4604F19800FFF7D6FE002004B010BD6C
:103B10000FB47FB5062102A8FFF7E6F8BDF8441000
:103B20009DF84040724D01AA002010800B0A8DF8CC
:103B300004308DF805104FF6FF76009602232146DB
:103B4000284602F0ADFC0096062302AA214628462C
:103B500002F008FD80B9FF2102A8FFF799FF02AC2F
:103B6000A17888420AD0FF210DF10B00FFF790FFEA
:103B70009DF80D10884201D0012022E09DF8082018
:103B800063781298139943EA022300EE103A00F08A
:103B90001DF89FED4E1ADFED4E1A40EE811AC0ED72
:103BA000001AE0789DF80C2042EA002200EE102A6C
:103BB00000F00CF89FED471A20EE811A81ED001AF3
:103BC000002004B070BC5DF814FB0000B8EE400AA1
:103BD000DFED410AC0EE200A704700002DE9F843EE
:103BE000C4B004460D46DFF80C9126A84946782259
:103BF000FDF7B6FA08A809F178017822FDF7B0FAC6
:103C00000027DFF8F48008A800EB8700079026AEB5
:103C100006EB8700069084B0414668462822FDF7EF
:103C20009FFA0FBCFFF774FF30B9012000F0F4F8E1
:103C30007F1C0A2FE7DB08E02C485C2102F08AFF9A
:103C4000411C842209F1F00033E002220A2126A857
:103C500002F0B2FF019002220A2108A802F0ACFF94
:103C60009DED010A0090DFED1D0A00F047F81F48A6
:103C700004DBDFED1B0A00F041F807D45C2102F001
:103C800069FF411C8B2209F59A7012E09DED000A34
:103C9000B5EE400AF1EE10FA04DBDFED120A00F097
:103CA0002DF80AD45C2102F055FF411C8C2209F545
:103CB000D670FFF700FE002004E00198206001208C
:103CC0000099296045B0BDE8F083000000002F4353
:103CD000000034C20000C84200FF7F47000020C23D
:103CE0000100AA420100C84200040048D88E000822
:103CF000C8280020748A000888000020B4EE600AFA
:103D0000F1EE10FA70470000134B036003F154000A
:103D1000086080211160704710B5002113A00F4C7E
:103D200000F04BF86060002117A000F046F820601A
:103D300010BD38B50A4C0B4D286803F001F9206816
:103D400003F0FEF8642000F067F84FF400710648B5
:103D5000FFF7B9F8F0E700009C1D0020282C002098
:103D6000F01F0020202100200008004830910008AA
:103D7000333D0008000000000000000000020000C9
:103D800000000000000000003C91000811800008C5
:103D900003000000000000008000000000000000A0
:103DA0000000000001460020842918BFC81C70478D
:103DB00080B503F030FB002002BD38B5044684B066
:103DC00060690D4600281CBFA069002812D0B4F914
:103DD0000800FFF7E7FFA16902912B466269019293
:103DE000009022692168606803F00AFA0390039842
:103DF00005B030BDB4F90800FFF7D4FF03A9019165
:103E000000902B4622692168606892B203F029FA7B
:103E10000128ECD00020EBE780B51921B0FBF1F0D0
:103E200000B9012003F0DDFA002002BDDFF86C00CC
:103E3000006800F4C060704710B5DFF86010B0F59E
:103E4000007F086800F4C0601DD1B0F5007F22D06B
:103E50000A68DFF84C30012060F34A220A60322001
:103E60001C68DFF840204443B4FBF2F0401C00E043
:103E7000401E4A69530501D50028F9D1486941051A
:103E800009D5032010BDB0F5806F04D00A68022068
:103E900060F34A220A60002010BD0000007000405C
:103EA000BC00002040420F002DE9FC47050066D011
:103EB000DFF82477DFF83067BC68D7F80C80287803
:103EC000C10604F00C0408F0030848D524B10C2CFA
:103ED00008BFB8F1010F2CD13868810702D5A86955
:103EE00000284CD0396808074EBF39687168090945
:103EF000286A01F0F001814206D200F032FB00286E
:103F00003DD100F006FA07E000F003FA24B9286A70
:103F100000F027FB002832D100F0ABFABA6800F0BD
:103F200097FADFF8BC06006800F098FB010016D095
:103F3000E9E1A86928B3396841F00101396003F06B
:103F400029FC81463868810707D403F023FCA0EBE5
:103F500009000328F6D30320D5E100F0DAF9287828
:103F6000C10755D5082C04D00C2C08BFB8F1030F9D
:103F700017D1386881034BD56868002848D10120E3
:103F8000C1E138684008400000F0D8F9814638683F
:103F90008107E4D503F0FEFBA0EB09000328F6D36C
:103FA000D9E76868B0F5803F04D1386840F48030C4
:103FB000386011E0B0F5A02F386806D140F48020B9
:103FC0003860396841F4803105E020F48030386091
:103FD000396821F480213960686860B103F0DAFB48
:103FE00081463868810313D403F0D4FBA0EB0900A9
:103FF0006528F6D3AFE703F0CDFB8146386881032F
:1040000006D503F0C7FBA0EB09006528F6D3A2E7AD
:104010002878810713D5042C04D00C2C08BFB8F1E4
:10402000020F22D13868410502D5E8680028A6D0E1
:104030007868296920F0FE4040EA016078602878BD
:10404000010742D56869002870682FD040F0010050
:10405000706003F09FFB80467068810735D403F0E1
:1040600099FB00F052F9F7D375E7E86878B1396841
:1040700041F48071396003F08DFB8046386841055A
:10408000D6D403F087FB00F040F9F7D363E7386834
:1040900020F4807000F052F9804638684105CED592
:1040A00003F078FB00F031F9F7D354E74008400003
:1040B000706003F06FFB80467068810705D503F0E0
:1040C00069FB00F022F9F7D345E72878410767D567
:1040D000B86DC1004FF000080AD4B86D40F08050B0
:1040E000B8654FF00108B86D00F08050009000985E
:1040F000DFF8F894D9F80000C10513D4D9F800000E
:1041000040F48070C9F8000003F044FB8246D9F8FF
:104110000000C10506D403F03DFBA0EB0A00032814
:10412000F5D318E7A868012804D1306840F00100F1
:10413000306010E00528306806D140F0040030609F
:10414000316841F0010105E040084000306031680D
:1041500021F004013160A86841F2893960B103F0AF
:1041600019FB82463068810713D403F013FBA0EBE0
:104170000A004845F6D3EEE603F00CFB82463068B1
:10418000810706D503F006FBA0EB0A004845F6D3ED
:10419000E1E6B8F1000F03D0B86D20F08050B865AB
:1041A0002878810621D5686A0028B0680ED040F0D2
:1041B0000100B06003F0EEFA8046B068810714D4C5
:1041C00003F0E8FA00F0A1F8F7D3C4E64008400095
:1041D000B06003F0DFFA8046B068810705D503F0D0
:1041E000D9FA00F092F8F7D3B5E6A86A002800F0F3
:1041F0008980022872D1F868EA6A00F003019142CE
:1042000001BF00F0700110312A6BB1EB021F1DD10C
:104210006A6B00F4FE41B1EB022F02BF00F078415F
:10422000AA6BB1EBC26F11D1EA6B00F4C00101F5CA
:1042300000115208B1EB425F08D1296C00F0C06058
:1042400000F100704908B0EB416F43D00C2C46D010
:104250003868410101D43868C1003FF590AE00F0E4
:104260006AF804463868810105D503F093FA001B0B
:104270000328F7D36FE6F868DFF87413EA6A08409A
:10428000296B1043491E40EA0110EA6B696B520822
:1042900040EA0120296C521E490840EA4250491E5A
:1042A00040EA4160A96B40EAC160F860386840F0BC
:1042B00080703860F96841F08071F96003F06AFA43
:1042C0000446386881011DD403F064FA001B0328FA
:1042D000F7D340E63868810114D4E7E70C2C3FF4AB
:1042E0004EAE00F028F804463868810105D503F089
:1042F00051FA001B0328F7D32DE6F868DFF8F41213
:104300000840F8600020BDE8F687A0EB080003280D
:104310007047386840F0080038603968286A21F032
:10432000F001014339607968E86921F47F4141EA8D
:10433000002179607047386820F08070386003F0A1
:1043400029BA2DE9F0410400884655D0DFF8A8626B
:10435000306800F00700404502D200F06FF84BD102
:104360002078DFF87452810706D5A068A96801F0AB
:10437000F001814200F076F82078C1072AD5606804
:10438000032802D129688A0108E0022802D129689D
:104390008A0303E00028296802D18A0702D42BE0AF
:1043A0004A0529D5A968890840EA8100A86003F078
:1043B000F1F90746A868616800F00C00B0EB810FC6
:1043C00008D003F0E7F9C01B41F289318842F1D3EC
:1043D000032031E02078810706D5A068A96801F0A4
:1043E000F001884200F03EF8306800F00700804598
:1043F00004D200F023F801D001201DE0207841070D
:1044000005D5AA68E06822F4E0620243AA60217838
:10441000080706D5A968206921F4605141EAC00166
:10442000A96000F026F8AA6800F012F8BDE8F04193
:104430006B48006800F012B9BDE8F0813168C90826
:1044400048EAC1013160306800F00700404570471C
:104450006A49C2F30312895C604A01F01F01C84037
:104460001060704704D2A96821F0F0010843A860E9
:10447000704770B5584A634B9068D6680025002194
:1044800010F00C0006F003065F4C03D00C2812D18C
:10449000012E1AD115682E0704D4524D2E68C6F38A
:1044A000032502E01568C5F30315584E56F825504C
:1044B00048B9294624E0042808BF214620D008280E
:1044C0001ED119461CE00C281AD1D06800F0030058
:1044D000022803D0032808BF1D4600E02546D16806
:1044E000D068D268C0F306204543C1F30210C2F37E
:1044F0004161401C491CB5FBF0F04900B0FBF1F1F3
:10450000084670BD35483E4A006813684049C3F309
:10451000022206E031483A4A006813683C49C3F376
:10452000C222895C01F01F01C840704710B50F22FC
:104530000260334A136803F003034360146804F015
:10454000F0048460136803F4E063C3601268D20867
:1045500002F4E06202612848026802F007020A6081
:1045600010BD7CB52B4E054630680024C10002D535
:10457000FFF75CFC0EE0306840F08050306031683E
:1045800001F0805100910098FFF750FC316821F054
:1045900080513160B0F5007F04D1802D0CD9A12D60
:1045A00009D304E0802D88BF032405D801D102245B
:1045B00002E0702D00D101240F480168C90844EAC7
:1045C000C1010160006800F00700A04201D0012095
:1045D00076BD002076BD000000100240BC00002027
:1045E000B80000209410024090100240007000407B
:1045F0008C809D01FCFFEEFE00200240EC8F000845
:104600000810024000127A000024F40034900008E0
:1046100048910008581002400248416802788A1800
:1046200042607047B000002000B500BF13009646FE
:104630009446103928BFA0E80C50FAD85FEA417CB4
:1046400028BF0CC048BF40F8042BC90728BF20F87A
:10465000022B48BF00F8012B00BD000078B50446CE
:104660001D481E4D87B0016841F40061016001A939
:10467000006800F40060009002A8009AFFF756FF5F
:10468000FFF748FF1649174B2960B0FBF3F0401EB7
:1046900040F2E73268600021EA602961A960A961FF
:1046A0002846FDF77DFA060012D12846FDF7C5FA27
:1046B00006000DD11920FEF75BFC102C07D200225A
:1046C00021461920FEF736FC0748046000E0012669
:1046D000304608B070BD0000601002407029002014
:1046E000002C014040420F00B80000200D4882B06D
:1046F000816841F001018160816801F00101009150
:104700000099026842F0805202600022006800F0C6
:10471000805000900F2100986FF0010002B0FEF76A
:1047200009BC00BF5810024010B5044610460A46A6
:104730000146204603F034F8204610BD603000EBFF
:104740008100006800F0F8407047603000EB8100A5
:10475000016821F000410A4302607047C06800F41C
:104760004060401E8041C00F704700F11403C80D27
:1047700010B500F00400C018090D01F01F01036816
:1047800007248C40A34302FA01F11943016010BDD4
:10479000F8B504460020002500900CB90120F2BDB8
:1047A00004F15406706828B92046FEF7FDFC00208D
:1047B000B060307021688868800004D58A68DFF8AE
:1047C0005C0202408A6021688868C00012D48A684E
:1047D000DFF84C02024042F080528A60DFF8441257
:1047E000DFF844220868B0FBF2F2521C520000923B
:1047F00000F036FB20688168C90008D4726842F076
:10480000100272600125B16841F00101B160816858
:1048100072688908D30600D4CA0700F181807368E2
:1048200023F4807343F0020373608068C00714D4DC
:10483000DFF8F821DFF8F83110681A68DFF8F47152
:104840003B6810431843C00707D4DFF8EC21136816
:10485000606823F47C130343136004F13002607E2C
:10486000536894F8207043EA4033E0681843A36823
:104870000343012F43EA074303D1606A401E43EA22
:104880004043A06A20B100F470701843E36A034308
:104890002768DFF8A801D7F80CC000EA0C00034332
:1048A000FB60C9072368986826D4000724D4DF6812
:1048B000DFF88C11D0690F40217E0743107847EA5A
:1048C000813747EA4007DF60107A01280FD123685B
:1048D0001F69D16810696FF38A070F435169074355
:1048E00090690F43074347F001071F6104E0206808
:1048F0000169490849000161206901282068016BAC
:1049000005D1E2690909521E42EA011101E00909D3
:10491000090101630120716860F30101716004E025
:10492000706840F01000706001252846F2BD064610
:10493000DFF80401046870472DE9F04105460E4692
:10494000FFF7F6FF286881684907904604F01F04C6
:1049500061D405F154073A78012A5CD00121DFF8CF
:1049600088253970904218BF002C03D0052C18BF41
:10497000092C4CD1284600F029FA010044D179686D
:10498000DFF86005014041F480717960DFF8DC03F5
:104990002968814200D11CB9786820F480107860C1
:1049A0007868C10446BFB86820F006000020B860EF
:1049B0004346286D0FF26151C162286D0FF2C55157
:1049C0000163286D0FF2C55141631C212A681160F3
:1049D0000020387032462868416841F0100141607B
:1049E0002868C16841F00101C160286800F14001F8
:1049F000286D00F0EDFD2A68DFF8F01493680B4095
:104A000043F00403936007E00021397004E00022C2
:104A100001203A7000E00220BDE8F081C0FFFF5F96
:104A2000C0FFFF7FBC000020400D030008000450C1
:104A300008010450080204500803045007C0F0FFA6
:104A4000F9BFFFFFF8B50646002006F154050F46F2
:104A5000009000242978012901D10220F2BD012013
:104A6000287030688168490700F1758179680629E6
:104A700010D2891E03290CD8DFE801F002040608D1
:104A80000C2107E0122105E0182103E04FF48071AA
:104A900000E0062100F13003880900F00C003A68BC
:104AA000C01801F01F0103684FF01F0C0CFA01FC45
:104AB000C2F3846223EA0C0302FA01F11943016094
:104AC000306882688168520731D409072FD4BA68E8
:104AD000B2F1004F08D139680022FFF746FE306876
:104AE000416941F0004106E03968FFF73EFE306859
:104AF000416921F0004141613068C1683A69042A86
:104B000016D060303B6800EB820C9748DCF8002040
:104B1000024003F0F8431343C9087A69480000F0E3
:104B200006008240134343F00043CCF8003076E0A7
:104B30000021FFF703FE40033068214604D1FFF750
:104B4000FDFDC0F3846003E0FFF7F8FD00F01BF902
:104B500039684A030EBFC1F3846191FAA1F1B1FA39
:104B600081F1884204D1306800220021FFF7EDFD79
:104B700000F016F9400304D100F012F9C0F384608C
:104B800003E000F00DF900F0FEF839684A030EBFAB
:104B9000C1F3846191FAA1F1B1FA81F1884204D1A3
:104BA000306800220121FFF7D0FD00F0F5F8400346
:104BB00004D100F0F1F8C0F3846003E000F0ECF8F9
:104BC00000F0E1F839684A030EBFC1F3846191FA3D
:104BD000A1F1B1FA81F1884204D1306800220221AA
:104BE000FFF7B3FD00F0D4F8400304D100F0D0F893
:104BF000C0F3846003E000F0CBF800F0C4F839683B
:104C00004A030EBFC1F3846191FAA1F1B1FA81F1B7
:104C1000884204D1306800220321FFF796FD3168F5
:104C20008868C00747D4FA683B68D1F8B0C0DFF89D
:104C3000C0E202F01802C3F312002EFA02F22CEACC
:104C4000000013400343C1F8B030F868DFF8A41245
:104C5000884230D1386841030EBFC0F3846290FAB5
:104C6000A0F1B1FA81F2521C012102F01F020A2ABE
:104C70000DD200F099F8920603F01F03401C02F0D9
:104C8000F842994000F01F0000F072F80FE000F0C9
:104C90008BF8401C920603F01F0300F01F0002F087
:104CA000F84299400A3800F063F841F00071BA68A0
:104CB0003068FFF75AFD3B68DFF83C0203424FD0F3
:104CC000DFF83802DFF838C20168DFF81C72DFF85D
:104CD0003422634501F0E0711ED10B0240D43368E9
:104CE000934218BFBB423BD100F048F841F40001A9
:104CF0000160DFF81402DFF814220168B1FBF2F260
:104D0000521C0C2042430092009800281EBF0098BD
:104D1000401E0090F8D123E0DFF8F4E173450BD199
:104D2000CB011DD43368934218BFBB4218D100F0A9
:104D300025F841F080710CE0DFF8D871BB420FD14B
:104D40004B020DD4366896420AD100F017F841F4B0
:104D50008001016004E0686840F020006860012480
:104D6000002028702046F2BD00F0FF03000104502F
:104D7000114300EB400041EA00517047026822F005
:104D8000E0721143704790FAA0F0B0FA80F07047DB
:104D900030680321FFF7D2BC30680221FFF7CEBC98
:104DA00030680121FFF7CABC420306D1C0F3846218
:104DB000C0F38463C0F3846005E090FAA0F0B0FA19
:104DC00080F213461046521C5B1C70477CB50446AB
:104DD0000020009021688868C20735D488686FF386
:104DE0009E1000282DD18868404D284040F00100D9
:104DF00088604249086800020AD54349434B0A6863
:104E0000B2FBF3F35B1C0C204343009300F028F843
:104E100002F0C0FC064620680168CA0714D4806806
:104E2000C00705D420688168294041F001018160F4
:104E300002F0B0FC801B0328EDD320680168CA078C
:104E4000E9D400F003F876BD002076BDA06D40F0F7
:104E50001000A065E06D40F00100E06501207047A2
:104E600002E00098401E009000980028F9D1704799
:104E700038B50446216888688A68D2072ED580072D
:104E80002CD48A6802F00D02012A1DD18A681748C5
:104E9000024042F002028A6003212068016002F0B1
:104EA00079FC054621688868C10717D502F072FCB5
:104EB000401B0328F6D320688168C807F2D5A16D8E
:104EC00041F01001A16503E0A06D40F01000A06565
:104ED000E06D40F00100E065012032BD002032BDF0
:104EE00000000000FEF1FFFF00020450C0FFFF7F42
:104EF000FFFF070000007F40000008800803045007
:104F0000000052C700000450BC000020400D030008
:104F1000000084CB0100008010B5846AA16D11F0FF
:104F2000500F22D1A06D40F40070A0652168086880
:104F30000207084606D5FFF711FC88B12068C16852
:104F4000880401E0C16888070AD4A16D21F480714A
:104F5000A165A06DC10403D4A06D40F00100A0655F
:104F60002046BDE8104002F024BCA16DCA0604D55D
:104F70002046BDE8104002F01DBC216D4A6BBDE823
:104F800010401047806A02F016BC0000806A816DF4
:104F900041F040018165C16D41F00401C16502F03D
:104FA00009BC00002DE9F84F064600253068DFF8FF
:104FB00050730105A84621D5B06E70B1B0F5800FD1
:104FC00017D0B0F5000F03D0B0F5400F09D013E0B3
:104FD0003A6842F480323A6004E0002100F08DF932
:104FE000054655B9F96FB06E21F440010143F967E8
:104FF00004E000F07CF9F3E70125A8463068C1041D
:1050000021D5F06EA8B1B0F1807F17D0B0F1007F4C
:1050100003D0B0F1407F04D013E0396841F480310F
:1050200039607DB9F96FF06E21F040710143F96785
:1050300009E0002100F061F90546F2E700F057F9B8
:10504000FAE70125A8463068DFF8B84281032ED57B
:10505000F86CC1004FF000090AD4F86C40F08050A1
:10506000F8644FF00109F86C00F08050009000984F
:10507000DFF894A2DAF8000040F48070CAF800006B
:1050800002F088FB8346DAF80000C10500F18B804E
:1050900002F080FBA0EB0B000328F4D30325A84605
:1050A000B9F1000F03D0F86C20F08050F86430782C
:1050B000C10705D5FA6FB06B920840EA8202FA6721
:1050C0003178880705D5F96FF06B21F00C010143A9
:1050D000F9673178480705D5F96F306C21F0300158
:1050E0000143F9673178080705D5F96F706C21F035
:1050F000C0010143F9673178C80605D5F96FB06C76
:1051000021F440710143F9673178880605D5F96FBC
:10511000F06C21F440610143F9673168880505D5D9
:10512000F96F306E21F440210143F9673168480579
:1051300005D5F96F706E21F440110143F96731789C
:10514000480605D5F96F306D21F440510143F967E8
:105150003178080605D5F96F706D21F4404101439F
:10516000F9673168C80505D5F96FB06D21F4403194
:105170000143F9673168C80205D5E168F06D890817
:1051800040EA8101E1603168880447D5F96F306FEA
:1051900021F040610143F967306FB0F1006F35D104
:1051A00000F0A0F83AE0002D7FF479AF206810F409
:1051B00040701EBF06F184014A6890420BD02068FF
:1051C000216841F48031216020F44070226822F48B
:1051D000803222602060C0070FD502F0DBFA05465E
:1051E0002068810709D402F0D5FA401B41F28931C9
:1051F0008842F5D34FF0030852E706F18402216894
:10520000506821F440710143216049E7B0F1806F9B
:1052100004D100F071F8010018BF80463068010326
:1052200014D5FA6F706F22F040620243FA67706F14
:10523000B0F1006F02D100F055F807E0B0F1806FD7
:1052400004D100F059F8010018BF804630684103CE
:1052500014D5FA6FB06F22F040620243FA67B06F64
:10526000B0F1006F02D100F03DF807E0B0F1806FBF
:1052700004D100F041F8010018BF804630684104B5
:1052800018D5FA6FF06F22F040520243FA67F06FC0
:10529000B0F1805F03D1022100F02FF807E0B0F1F8
:1052A000005F07D1022106F1200000F0A2F8010002
:1052B00018BF80463068010406D5FA6FD6F8800022
:1052C00022F080420243FA673168C80306D5F96FBD
:1052D000D6F8840021F000410143F9675FFA88F0B5
:1052E000BDE8F28F386840F48010386070470021C4
:1052F00006F1200000F07DB80121301D00F006B855
:105300000C10024090100240007000402DE9F04166
:105310000546794F28680C46F968002611F0030FFE
:105320000DD0F96801F00301814231D180B3F868F2
:105330006968C0F30210401C88420ED028E00128A2
:1053400004D025D303281DD018D321E03A68910753
:105350001ED5FA68696800F0C3F8386820F08060EC
:1053600000F0C6F880463868010113D502F012FA41
:10537000A0EB08000328F6D3032637E039684A0576
:10538000E7D405E039688A03E3D439684A03E0D4F6
:1053900001262BE0A9682CB93A695848EB6800F05F
:1053A0008FF80FE0012C3A6909D12B69544802406B
:1053B0005B0842EA01215B1E41EA435102E06B694E
:1053C00000F084F83961386840F0806000F090F8AF
:1053D00004463868010105D402F0DCF9001B0328FB
:1053E000F7D3C9E73869A969084338613046BDE891
:1053F000F0812DE9F04106463F4F30680C46F968D0
:10540000002511F0030F0DD0F96801F0030181426E
:1054100031D180B3F8687168C0F30210401C884233
:105420000ED028E0012804D025D303281DD018D39E
:1054300021E03A6891071ED5FA68716800F050F8CB
:10544000386820F0805000F053F8804638688100BA
:1054500013D502F09FF9A0EB08000328F6D303252B
:105460002BE039684A05E7D405E039688A03E3D4BC
:1054700039684A03E0D401251FE0B1687A69002C3D
:1054800004D11E48F36800F01BF802E0336900F015
:105490001DF87961386840F0805000F029F8044622
:1054A0003868810005D402F075F9001B0328F7D392
:1054B000D5E778697169084378612846BDE8F081CD
:1054C000024042EA012141EAC36170470D480240AF
:1054D0005B0842EA01215B1E41EA4361704700001C
:1054E00022F073021043491E40EA0110F860704731
:1054F000386002F04FB9000000100240FF80FF0743
:10550000FF809FFFFF80FFF970B508B9012070BDD3
:105510000268284D284CAA4200F1240308D22749EA
:105520008A181426B2FBF6F292001A62DC6108E0D7
:1055300023498A181425B2FBF5F2920021491A6218
:10554000D96102225A7001680D688168C2680668D4
:105550006FF30E150D430169154342690D438169CF
:105560001543C2690D43016A15430D4335608268D6
:10557000B2F5804F17D0DA690F21A2420CBF124A50
:10558000124A146893F8205005F01C05A94024EA3B
:1055900001011160116893F82040406804F01C0478
:1055A000A0400143116000209861012159701870DA
:1055B00070BD00000804024000000240F8FFFDBF7B
:1055C000F8FBFDBF00040240A8000240A80402400E
:1055D000F8B5044604F1240600253078012801D1ED
:1055E0000220F2BD012030707778012F26D10220F1
:1055F00070700027B7612068D0F800C04FEA5C07E0
:105600004FEA470CC0F800C0204600F0C4F82168FB
:10561000F06820B10A6842F00E020A6008E00868EB
:1056200020F0040008602068016841F00A01016070
:105630002068016841F00101016001E03570022538
:105640002846F2BD00F124014A78022A05D0042040
:10565000886100220A70012070470268136823F0F5
:105660000E031360006802685208520002600120B5
:1056700091F82020CB6902F01C0290405860002273
:10568000012048700A700020704738B500F12401ED
:1056900000244A78022A03D004208861012417E0FC
:1056A0000268136823F00E031360026815686D0822
:1056B0006D001560012291F82030CD6903F01C03C4
:1056C0009A406A6001224A700C70496901B18847AA
:1056D000204632BDF8B500F124010423CA691468DC
:1056E0000268156891F8206006F01C0603FA06F7B8
:1056F0003C4210D06F070ED51468A50603D4146879
:1057000024F00404146000F03EF8C968002939D080
:10571000BDE8F4400847022303FA06F73C4213D0E1
:10572000AF0711D51468A50605D4146824F00A043F
:10573000146001224A7000F026F800220A7089687D
:1057400001B3BDE8F4400847082303FA06F63442E3
:1057500018D02B0716D5146824F00E04146001220B
:1057600091F82030CC6903F01C039A406260012359
:1057700001228A614B7000220A70096911B1BDE8EB
:10578000F4400847F1BD91F82020CC6902F01C02DA
:1057900093406360704770B590F84450066C0124E4
:1057A00005F01C05AC4074600468636080681028D4
:1057B00002D1A260E16070BDA160E26070BD2DE920
:1057C000F04104000D461646984608BF012034D02B
:1057D00004F17807786820B9002139702046FDF778
:1057E000B2FD242078602068016849084900016002
:1057F000606A10B1204600F069FB204600F052FAC2
:1058000001281AD02068816841F4804181602068B5
:10581000816821F400410D438560206801686FF3C1
:10582000194141EA465141EA0841016000F007F898
:105830002046BDE8F04100F0ACBBBDE8F081206837
:10584000016841F0010101607047000038B50400B3
:1058500001D1012032BD04F17805686808B900F073
:1058600017F800F01AF808B100F031F800F02CF841
:10587000012804D000F004F821F02A0116E032BD1E
:105880002068416821F49041416020688168704738
:10589000002129702046FDF756BD2420686020684D
:1058A0000168490849000160606A7047816000F042
:1058B00004F8BDE8324000F06CBB2068016841F09C
:1058C0000101016020467047204600F0EBB92046F8
:1058D00000F0FCBA2DE9F843054605F150060C46E8
:1058E000F06A2028174699463ED10CB1380001D104
:1058F00001203AE0002070632121F16201F04AFFAB
:10590000378080467780A868B0F5805F04BF28693B
:1059100000281ABF204600272746044611E000222F
:10592000802100F024F8D8B92868002C12BF14F8A0
:10593000011B37F8021BC1F3080101857088411E65
:10594000718043467088CDF800900028E7D100228E
:10595000402100F00CF818B92020F062002004E08B
:105960002020F062032000E00220BDE8F2832846F8
:1059700000F05CBB38B50346D3F8800020280AD17C
:1059800009B1100001D1012032BD00F006F8BDE8D8
:10599000384000F091BB022032BD00201866DFF8CD
:1059A00000431868A0420CD04068040209D518686A
:1059B00050E8004F054644F0806445E80040002868
:1059C000F5D118467047286800F1080151E8001F1A
:1059D000490800F10803490043E800100028704717
:1059E000F8B5054640F60F0C2A68D369104613EA4D
:1059F0000C0F0668976805F1580406F0200003F0C4
:105A000020010BD1002918BF00280ED021690029E0
:105A100000F028812846BDE8F44008475FEAC77CCB
:105A200004D4DFF8A4E416EA0E0F78D05FEAC37C52
:105A300048BF5FEAC65E07D54FF0010CC2F820C030
:105A4000E26A42F00102E2629A070AD5FA0708D533
:105A5000D5F800E00222CEF82020E26A42F00402EB
:105A6000E2625A070AD5FA0708D5D5F800E0042201
:105A7000CEF82020E26A42F00202E2621A070BD559
:105A800008B9FA0708D5D5F800C00827CCF8207067
:105A9000E26A42F00802E2621A0509D5730107D5ED
:105AA0002E684FF400623262E26A42F02002E26243
:105AB000E26A002A32D0002918BF002803D02169E9
:105AC00009B128468847E06A29688A68510602D4E5
:105AD00010F0280F1DD0284600F048FB2868816888
:105AE000480611D500F0C9F8FCD1E06960B10FF2A9
:105AF000F5618163E069FFF7C8FD00280ED0E06919
:105B0000816BBDE8F44008472846BDE8F24001F04B
:105B100053BE284601F050FE0020E062F1BDA068AF
:105B2000012875D1D80673D5F10671D51020106201
:105B300029688868410639D5E1690868406880B2FB
:105B40000028EBD022889042E8DA6080086801687B
:105B50008A0623D400F09FF821F4807100F062FAE5
:105B6000F8D1FFF730FFFCD1286800F1080151E8B7
:105B7000001F00F1080321F0400100F07AF8F3D192
:105B80002020A0620021A16000F085F821F0100122
:105B900000F048FAF8D1E069FFF754FD0220E06018
:105BA00021886088091A89B228462DE021886288F8
:105BB0006088891A00281CBF88B2002852D02A4663
:105BC000106850E8003F054623F4907300F04BF84E
:105BD000F6D100F000FB00F108065B0046E800305B
:105BE0000028F6D12020A0620023A360236113685F
:105BF00053E8003F156823F0100300F034F8F6D1A5
:105C00000220E06089B21046BDE8F44001F0D5BD45
:105C1000D80209D5790207D54FF4801010622846C2
:105C2000BDE8F24001F0CABD180607D5310605D51A
:105C30006169B9B12846BDE8F4400847580611D556
:105C400071060FD500F027F821F0400100F0EAF9C5
:105C5000F8D120206062002161612846BDE8F24051
:105C600001F0ADBDF1BD45E800300028704721F0DE
:105C7000800143E8001000287047296801F10802FC
:105C800052E8001F286800F1080321F0400143E8B2
:105C9000001000287047286850E8001F024670472F
:105CA00000800040F8B50446DFF8840622681368D7
:105CB000A168034020690B4361690343E0690B431A
:105CC0000343136000255168E06821F4405101430B
:105CD0005160A369DFF854168A421CBF206A03434F
:105CE0009668DFF85076DFF8500626F430663343C6
:105CF0009360BA424FF40043DFF8406632D1366811
:105D000006F00306032E3BD8DFE806F0027161843B
:105D10000127E169B1F5004F4FF6F07640F0AB8016
:105D20005FB1012F00F09F80022F0AD0042F00F0F6
:105D30009D80082F00F09D80BFE0FEF7E3FB002868
:105D40000FD061684A0802EB4002B2FBF1F0A0F10B
:105D50001001B142F0D20640C0F342000643206871
:105D6000C660ABE0DFF8D875BA4221D1366816F0CC
:105D70000C0660D0042E3AD0082E28D00C2E49D024
:105D800010278A42C5D137B1022F08D0042F54D032
:105D9000082F55D091E0FEF7B5FB0028E1D06268EE
:105DA00002EB4201884202D3130383424AD284E0C9
:105DB000DFF89075BA420CD1366816F030063AD04A
:105DC000102E14D0202E02D0302E23D0D8E7022758
:105DD000D7E7DFF87475BA420BD1366816F0C00603
:105DE00029D0402E03D0802EF1D0C02EEDE704271D
:105DF000C7E7DFF85875BA420ED1366816F4407618
:105E000019D0B6F5807FF2D0B6F5007FDFD0B6F5B9
:105E1000407FB5D10827B4E78A42B1D1366816F47D
:105E2000406608D0B6F5806FE1D0B6F5006FCED0F1
:105E3000B6F5406FC9E70027A3E7FEF71AFBACE70A
:105E40001846ACE7010E560816EB00206941002306
:105E5000FBF714FEA0F54071DFF8F42491422CD238
:105E60002168C8602AE0FEF755FB68E7FEF701FBF2
:105E700065E7184665E747B1012F16D0022F07D016
:105E8000042F15D0082F16D017E0FEF73BFBA8B162
:105E9000616800EB5100B0FBF1F0A0F11001B142DC
:105EA0000BD2226880B2D06008E0FEF733FBEEE749
:105EB000FEF7DFFAEBE71846EAE701250020A066C7
:105EC000E0662846F2BD00002001000490F824108E
:105ED0000A0706D502685368416B23F400430B435D
:105EE000536090F82410CA0706D502685368816A87
:105EF00023F400330B43536090F824108A0706D52F
:105F000002685368C16A23F480330B43536090F8EE
:105F100024104A0706D502685368016B23F48023D6
:105F20000B43536090F82410CA0606D502689368A4
:105F3000816B23F480530B43936090F824108A06FE
:105F400006D502689368C16B23F400530B4393603A
:105F500090F824104A0610D502685368016C23F4A7
:105F600080130B435360036CB3F5801F05D1536856
:105F7000416C23F4C0030B43536090F824100A06CD
:105F800006D501684A68806C22F4002202434A6008
:105F90007047F8B5054605F178040020E0606FF021
:105FA0007E4701F0F7FB0646286801680A0711D50D
:105FB0000097334600224FF40011FFF7D8FC48B198
:105FC000FFF769FE21F0800100F02CF8F8D12020C5
:105FD000606017E0286801684A0717D500973346C4
:105FE00000224FF48001FFF7C2FC78B1FFF753FEA7
:105FF00021F4907100F016F8F8D1FFF7E4FCFCD121
:106000002020A060002121700320F2BD20206060CC
:106010002021A16000202866002169662070F2BD61
:1060200021F4F07142E80010002870472DE9F0419A
:10603000069C05460E4690461F462868C1693140B9
:10604000B1420CBF01200020404533D114F1010FB3
:10605000F3D001F09FFBC01B844200D314B903208E
:10606000BDE8F081286801684A07E6D5C1690807DC
:1060700004D42968C8690105DFD50DE02A68082025
:106080001062284600F072F805F178000821C1601E
:10609000002202700120E3E729684FF400600862E3
:1060A000284600F063F805F178002021C160002245
:1060B0000270D4E70020D3E720B5034600205965DD
:1060C00003F158010A804A800861FF229868B0F500
:1060D000805F04D1186990B940F2FF120FE018B93F
:1060E000186960B17F2007E0B0F1805F06D11869C0
:1060F00008B97F2203E03F20888001E000228A80E7
:106100000020C86222228A62186800F1080252E860
:10611000002F00F1080542F0010245E800200028A8
:10612000F2D19868B0F5805F04BF186900280DD1DE
:106130000FF215120A61186850E8001F024641F07C
:106140002001FFF76FFFF6D1002020BD0FF2A9025A
:106150000A6118690028EED0196851E8001F1A6812
:1061600041F49071FFF75EFFF6D1EDE710B500F056
:106170000EF8FCD100F015F8FCD1016E00F01EF80D
:106180002021C0F8801000220266826610BD0168DE
:1061900051E8002F0B4622F4907243E800210029B9
:1061A0007047016801F1080252E8002F520801F11E
:1061B0000804520044E8002100297047012909D150
:1061C000026852E8002F036822F0100243E8002121
:1061D0000029F5D17047106800F1080353E8003F2B
:1061E0005B087047806A00F1520100220A81002397
:1061F0000B8001F0E1BA000038B500F04DF81ED177
:106200008B8C9188446D0B402370416D4B1C00F0CA
:1062100049F818D100F04DF800F060F8FCD100F01A
:106220006AF80BD10023936000F04EF8FCD10168AE
:10623000CB69DC0644BF10230B628BE08FE0088B38
:1062400040F00800088331BD38B500F025F81ED1B4
:106250008B8C9188446D0B402380416D8B1C00F02A
:1062600021F818D100F025F800F038F8FCD100F042
:1062700042F80BD10023936000F026F8FCD10168AE
:10628000CB69DC0644BF10230B6263E067E0088B38
:1062900040F00800088331BD00F158020168936A9C
:1062A000222B7047436551884B1E5380518800292B
:1062B0007047036853E8003F046823F4907344E890
:1062C00000310029F5D17047016851E8003F0C46C4
:1062D00023F0100344E8003100297047016801F100
:1062E000080353E8003F5B0801F108055B0045E83F
:1062F00000310029704720219162002313610021A1
:10630000D1600A4B016899420CD049680B0209D54B
:10631000016851E8003F0C4623F0806344E80031F7
:106320000029F5D1916801297047000000800040E4
:10633000F369FFEF003801400024F40088100240A8
:106340000044004000480040004C00400050004025
:1063500000FD0F001188BDE8344001F02EBABDE801
:10636000324001F02DBA000030B500F14002537800
:10637000202B0CD11478012C09D000F01DF824F446
:1063800080541C6003681D682943196020E00220C6
:1063900030BD30B500F140025378202B0AD114787B
:1063A000012C07D000F008F824F4706444EA0124BA
:1063B0001C600DE0022030BD0123137024245470B2
:1063C00003681D686D086D001D6003681C687047D8
:1063D0000068016841F00101016020205070002137
:1063E0001170002030BD000038B5040001D101203B
:1063F00032BD04F14005687820B90021297020469B
:10640000FDF7F3F800F044F86068216820F0706050
:1064100008612068816821F400418160E0680128FA
:10642000A0680CBF40F4004040F40440216888603C
:10643000E0680228206841680CBF41F4006121F443
:10644000006141602068416841F0007141F4004101
:1064500041602068C16821F40041C1606069216920
:10646000A2690143206841EA0221C160206AE16912
:106470002268014311602068016841F00101016058
:10648000002068602021697020630021A97032BD5E
:10649000242068702068016849084900016070473D
:1064A0002DE9F84300F0B5F859D12178012956D0EB
:1064B0000120207001F06EF900F0DEF800284CD1C8
:1064C000212000F0AFF8708DDFF81012B0F5807F5A
:1064D00003D335854FF0807304E0708D30854FF025
:1064E000007390B1706AD6F800C00278CCF828200A
:1064F000706A421C7262708D421E7285308D421E1F
:1065000032850091521CD2B204E00091002201E0D9
:1065100000F0BCF800F0A4F800F075F818D000F016
:106520001BF9002819D100F08CF80028F4D089B2AA
:106530000029F1D100F098F878B900F07EF8E7D2A0
:10654000708D3085002100914FF00073328DDAE7B5
:1065500000F02FF900F0A1F802D0012000E00220A5
:10656000BDE8F2832DE9F84300F053F843D12178D8
:10657000012940D00120207001F00CF900F07CF8D6
:10658000002836D1222000F04DF8718DDFF850013F
:10659000B1F5807F28BF358509D2718D3185009096
:1065A0004FF00073328DD2B203E03585002000F049
:1065B00025F800F055F800F026F815D000F01AF98B
:1065C000002816D100F07BF80028F4D089B2002909
:1065D000F1D100F049F860B900F02FF8E5D2708DE4
:1065E000308500210091DBE700F0E3F800F055F87A
:1065F00002D0012000E00220BDE8F28300904FF0BD
:106600008073FF227047708D00284A463946304615
:106610007047064606F140048846607820281546F3
:106620001F46704760701021A17000206060756285
:1066300077857063FF25089F7047708DB0F5807F68
:106640007047706A326801789162706A411C7162A9
:10665000708D411E7185308D411E3185708D704762
:106660004146304600F089B9CDF800903B46002203
:106670008021304600F046B88146CDF800901923BD
:1066800001224FF40041304600F03CB8358500202F
:1066900000904FF08073FF22704701000DD13268E7
:1066A0002020D0613268DFF83C005368034053601B
:1066B000202262700020A0702070080070473068AF
:1066C000416A706A0170716A308D4A1C411E7262A3
:1066D0003185708D421E7285708D7047002000805C
:1066E0000024008000E800FE006881698A0744BF3A
:1066F000002181628169CA0703D4816941F00101E7
:10670000816170472DE9F041069F05460E4690468F
:106710001C46286881693140B1420CBF012000202D
:10672000404517D114F1010FF3D001F033F8C01B2D
:10673000844201D3002CECD1286881693140B142F8
:106740000CBF012000204045E3D100F026F80120D5
:10675000BDE8F0810020FBE770B505460C46164603
:1067600028688169880716D400F040F818B914F138
:10677000010FF5D001E0012070BD01F00BF8801B86
:10678000844201D3002CEBD1286881698807E7D4C3
:1067900000F003F8EFE7002070BD05F14000202273
:1067A000416841F020014160427000218170017018
:1067B000704770B505460C461646286881698806FC
:1067C00012D400F013F808B1012070BD00F0E2FF10
:1067D000801B844201D3002CEFD128688169880690
:1067E000EBD4FFF7DAFFEFE7002070BD3246214619
:1067F000284647E070B505460C461646286881696C
:1068000048073DD4FFF7F2FF002837D12A68906986
:1068100081061ED59069410701D5288D80BB9069FE
:10682000C30605F1400104D51020D06104224A605E
:1068300001E00020486020222868C2612A68584888
:1068400053680340536020224A700020887008700B
:1068500014E000F09FFF801B844201D3002CCDD1B7
:10686000286881694807C9D405F1400020224168A1
:1068700041F020014160427000210170012070BD93
:10688000002070BD2DE9F843044600252068836987
:1068900000269046DA0604F1400739D51023C3617B
:1068A00089462BE029002DD119F1010F26D000F0E7
:1068B00071FFA0EB0800814502D3B9F1000F1DD193
:1068C00020684168BA7883691B040AD5490408D452
:1068D000202A06D0416841F48041416000F05AFF0F
:1068E000804620688169880608D400F053FFA0EB39
:1068F00008001A28F5D346F0200601252068816992
:106900008A06CFD50DB92021C16146F004060125C4
:1069100020688169CA0505D54FF4807346F00106E9
:10692000C3610125480506D520684FF4806246F012
:106930000806C2610125880507D520684FF400715B
:1069400046F00206C161012501E028000CD0204676
:10695000FFF7CAFE00F00BF8202079680E437E6036
:1069600078700021B97039702846BDE8F28321683B
:106970000B484A6802404A60704770B50068049C42
:106980004568084EC1F3090141EA0241194346EA4C
:1069900054562143B54321F000412943416070BD65
:1069A00000E800FEFF63FF0338B5040001D10120B9
:1069B00032BD606A30B96068B0F5827F05D00021D1
:1069C000E16102E00020206160610020A06204F12A
:1069D0005C05687820B9002129702046FCF7B6FED6
:1069E0000220687000F04AF8E168B1F5E06F04D960
:1069F0000020B1F5706F03D104E04FF4805001D056
:106A00000021A1626168A268237C01F4827102F412
:106A100004421143227D03F002031943A36902F0EB
:106A200001021143227F03F40073194394F82030CC
:106A300002F038021143A26A03F08003194323686D
:106A400002F4005211431960A16994F8242094F8CB
:106A50003430090C01F0040102F010021143E26825
:106A600003F00803194302F47062114308432168DC
:106A70004860002068600121697032BD20680168AB
:106A800021F0400101607047016042600021C16057
:106A9000002282600120704710B5C2684368521C12
:106AA00092FBF3F403FB142283689A4202D16FF045
:106AB000010010BD0268C368D154C16800F014F829
:106AC000C160012010BD10B58268C3689A4201D12F
:106AD000002010BD02688368D45C0C70816800F0EF
:106AE00003F88160012010BD4268491C91FBF2F35C
:106AF00002FB13117047000037B5044600250A4613
:106B00000194009502AB01A9074878441A30F9F7BF
:106B100050FB019A157000284EBF04460198041BD3
:106B2000204603B030BD00BF83A5FFFF38B5044643
:106B300000F030FE14F1010F054602D00448017840
:106B4000641800F027FE401BA042FAD331BD00BFFD
:106B5000B00000200246C9B2002013788B4205D055
:106B600012F801CBBCF1000FF7D170471046F7E7E0
:106B7000C0F3C75181B1FF2906D0C110400721F0F1
:106B8000E04101F16051704741020CBF40F4E00167
:106B90006FF000410020704700F0004100020AD071
:106BA000B0FA80FC00FA0CF001F16051A1EB0C513D
:106BB00001EBD02140057047F8B5D2B2022A3CD192
:106BC000C9B200244A1E18E000EB860500EB8607D8
:106BD00095ED010AD7ED000AB4EE600AF1EE10FA65
:106BE00005D5CDED000A87ED000A009F6F60761C89
:106BF0000D1B6D1EAE42E7DB641C9442B8BF00263D
:106C0000F6DB012400930AE000EB83039DED000A0C
:106C1000D3ED000A70EE200ACDED000A641CE3B249
:106C20009342F1DB891E00EE101AB8EEC00ADDEDCA
:106C3000000AC0EE800ACDED000A0098F2BD000007
:106C400030B503464FF6FF70002400E0641CE2B24A
:106C50008A4211D213F8012B5040082205046D0C12
:106C600000F001000128B2BF284685F4204080F0E2
:106C70000100521EF2D1E9E730BDDFF808040168D7
:106C800002E0DFF80004416800EE101AF2EE040A98
:106C900020EE200ABDEEC00A10EE101A0804000E05
:106CA00040EA012080B27047DFF8D8038168EBE743
:106CB000DFF8D003C168E7E7DFF8C8030169E3E75D
:106CC000DFF8C0034169DFE7DFF8B8038169DBE77C
:106CD000DFF8B003C169D7E74FF4006070474FF4A5
:106CE000106070474FF420607047DFF89C034078D5
:106CF00000027047F8B50446DFF8907315461E464B
:106D00003221384600F05EFDDFF87C235078387081
:106D100003217970BE7032462946F81CFAF720FA32
:106D2000B978C91CC9B23846FFF78AFFF91C8853E5
:106D300039462046BA78BDE8F840521DFCF78EBDB2
:106D400020B50021DFF848238BB252F83350A84217
:106D500004D0491C8BB20C2BF6D306E002EBC30126
:106D600000204A68BDE820401047002020BD0000F8
:106D70002DE9F84380460C46DFF81893C8214846B1
:106D8000FBF7B2FFA278E57820796679C24C45EA34
:106D90000225642D46EA002608DB00F0A4F8411C19
:106DA0002B464FF4897204F1300009E0642E08DBB1
:106DB00000F099F8411C334640F2131204F19000A0
:106DC00095E000F089F880B900F08DF8411C4FF48F
:106DD0008B7204F1E400FCF76EFD9FEDA90A10EE42
:106DE000100AB86110EE101AF961002406E060196B
:106DF000C0B2FFF7A5FF29F81400641CB442F6DB0B
:106E0000A6480168884508BF00F0E4F8A448016876
:106E1000884509D173009BB24A4603214046FFF7DB
:106E200069FFBDE8F143D5E0BDE8F1832DE9F84302
:106E300080460C469EA0DFF86C92FCF73CFDC82112
:106E40004846FBF751FFA078E578667945EA0025CA
:106E50002079914C642D46EA002608DB00F043F8C7
:106E6000411C2B464FF49D7204F1300009E0642E62
:106E700008DB00F038F8411C334640F23B1204F1C5
:106E8000900034E000F028F880B900F02CF8411CA4
:106E90004FF49F7204F1E400FCF70DFD9FED780ABA
:106EA00010EE100AB86110EE101AF96100F092F8B5
:106EB000002406E06019C0B2FFF742FF29F8140071
:106EC000641CB442F6DB4A46404601B07300BDE89C
:106ED000F0439BB203210DE76A4F07F11C0107F154
:106EE0001800FCF77BBE5C212046FFF733BE01B0E3
:106EF000BDE8F043FCF7DFBCF8B50D460446911E33
:106F0000C9B22846FFF79CFEA979EA7941EA022135
:106F1000884214D16878032818BF10280FD10026A2
:106F2000614F687857F83610884205D107EBC602E2
:106F30002946536820469847761C022EF1D3F1BDAE
:106F400078B58DB00546FCF798FC00283FD014209A
:106F5000FCF762FF554C32212046FBF7C5FE0026A8
:106F60002846FCF797FCA055761C312EF8D34649ED
:106F70004B780020225C9A4205D1621C125C032AE5
:106F800018BF102A03D0401C3128F3D31FE031284A
:106F90001DD0C0F1310221186846FAF7E1F89DF8DA
:106FA0000100032805D1082221462846FFF7A4FF47
:106FB0000DE0102840F00B809DF806403EA52146CC
:106FC0002846FCF778FCE11D2846FCF774FC0EB05F
:106FD00070BD000010B52B4C2068FFF7C9FD0246BC
:106FE0004FEA010336A0FCF766FC6068FFF7C0FDBE
:106FF00002460B463AA0FCF75EFCA068FFF7B8FD1E
:1070000002460B463EA0FCF756FCE068FFF7B0FDD9
:1070100002460B4642A0FCF74EFC2069FFF7A8FD94
:1070200002460B4646A0FCF746FC6069FFF7A0FD50
:1070300002460B464AA0FCF73EFCA069FFF798FD0C
:1070400002460B464EA0FCF736FCE069FFF790FDC8
:1070500002460B4652A0FCF72EFC206AFFF788FD83
:1070600002460B4656A0FCF726FC606AFFF780FD3F
:10707000BDE8104002460B4659A0FCF71CBC0000BE
:1070800000000000F02B0020700000206428002089
:107090001000002050220020988C0008F01F0020D3
:1070A000202100201823002000000020BC2B0020FD
:1070B000303030303000000025640D0A0000000040
:1070C0006D696E5F77696E645F6469726563746928
:1070D0006F6E3A202020202020252E32660D0A00D7
:1070E000617665726167655F77696E645F64697216
:1070F000656374696F6E3A2020252E32660D0A0092
:107100006D61785F77696E645F64697265637469E5
:107110006F6E3A202020202020252E32660D0A0096
:107120006D696E5F77696E645F73706565643A2040
:10713000202020202020202020252E32660D0A002D
:10714000617665726167655F77696E645F737065AC
:1071500065643A202020202020252E32660D0A006A
:107160006D61785F77696E645F73706565643A20FE
:10717000202020202020202020252E32660D0A00ED
:1071800074656D70657261747572653A2020202097
:10719000202020202020202020252E32660D0A00CD
:1071A00068756D69646974793A2020202020202058
:1071B000202020202020202020252E32660D0A00AD
:1071C00070726573737572653A202020202020202C
:1071D000202020202020202020252E32660D0A008D
:1071E0007261696E3A20202020202020202020205B
:1071F000202020202020202020252E32660D0A006D
:10720000F0B585B050260B9D25B986F3118800F0A6
:1072100019FAFEE70C9C24B986F3118800F012FAE3
:10722000FEE754270097DDF800E0BEF1540F04D0CC
:1072300086F3118800F006FAFEE7009E256300261B
:10724000022584F8515004AF0A9D039602940197D9
:10725000009500F034F8204600F06FF8049805B06F
:10726000F0BD2DE9F8430646174684B08846994696
:10727000B80000F0ABFA05001CD0542000F0A6FACC
:10728000040014D00020256384F851000390029478
:107290000D980C99019000914B463A464146304674
:1072A00000F00DF8204600F048F8012004E02846E0
:1072B00000F014FB4FF0FF3005B0BDE8F0832DE97E
:1072C000F0470A9E8046306B00EB8202101FC00818
:1072D0004FEAC00A06F1340451B100228D5CA55476
:1072E000885C10B1521C102AF8D30020E07300E033
:1072F0002170089F062F88BF0627099DF762276126
:10730000002161619946301D00F045FB06F118002F
:1073100000F041FB3661C7F10707B76176620020D4
:10732000A061002121774A464146504600F070FB9B
:10733000306005B12E60BDE8F0872DE9F04100F026
:1073400067F8DFF8BC53DFF8BC83E86C401CE864E6
:107350001426A86A28BBAC62E86C012829D1002752
:1073600006FB07F0404400F009FB7F1C072FF7D312
:1073700005F1740000F002FB05F18807384600F0C3
:10738000FDFA284600F0FAFA05F1140000F0F6FACA
:1073900005F1380000F0F2FA05F17400E8622F639D
:1073A00007E0A86D28B9E06AA96ACA6A904228BFB6
:1073B000AC62A86E401CA86600F096F94643211DF9
:1073C00008EB060000F0EAFA00F0ADFBA86D30B162
:1073D00000F03DF903D200F09AF900F033F9BDE86E
:1073E000F08180B588B1DFF81823116F21B100F06A
:1073F0003CF800F027F9FEE7116F491C11670021E6
:1074000000F08BF900F03BF808B900F016F901BD67
:10741000044600F06FBB80B586B000210591049151
:1074200003AA04A905A8FCF76FFC0598049902902B
:107430000022009201910023039A0FF250310FF2C3
:107440001920FFF7DDFE70B100F00FF800F0FAF838
:10745000DFF828034FF0FF31C16601228265002169
:10746000016500F0F7FA07B000BD502080F31188E5
:107470007047DFF80803016F491C0167704770B55A
:10748000DFF87C62306F0024002520B900F044F85A
:1074900000F0D8F8FEE700F02DFB306F401E30679B
:1074A000306F002837D1F06CD8B934E0F068C46888
:1074B00000F036F800F015F9E06A716DDFF8B832C7
:1074C000012282401143716514225043211D18444A
:1074D00000F064FAE06AB16ACA6A904224BF0121EE
:1074E000316630680028E1D10CB100F0EDF8F46DA0
:1074F00044B100F019F808B101203066641EF8D1DB
:107500000020F065306E30B1DFF874124FF080501B
:10751000012500F096F8EEE0502181F311887047C4
:1075200004F1180000F060BA2DE9F843DFF8D071DB
:10753000386F0026002853D13C6D641C3C6510D187
:10754000F86A006820B1FFF7E7FF00F07BF8FEE77C
:10755000F86A396BF9623863786E401C786600F01F
:10756000B3F8F86EDFF8109284424FF0140828D375
:1075700020E0F96AC868C568686884422ED3281D6F
:1075800000F032FAA86A18B105F1180000F02CFAE0
:10759000E86A796D012282401143796508FB00F0A9
:1075A000291D484400F0FAF9E86AB96ACA6A9042AB
:1075B00028BF0126F86A00680028DAD14FF0FF31B1
:1075C000F966B86AC06A08FB00F859F80810022981
:1075D00028BF0126386E30B1012604E0F866F0E7D6
:1075E000F86D401CF8658FE0DFF81421106F10B1C2
:1075F00001211166704710661421506DB0FA80F3B6
:10760000C3F11F034B43DFF87011C85838B950213C
:1076100081F31188BFF34F8FBFF36F8FFEE7C81858
:1076200000F10803416849684160994204BF496814
:1076300041604068C16891627047DFF844114FF0C3
:1076400080500860BFF34F8FBFF36F8F7047A86AF9
:10765000C16AE06A8142704770B5DFF8A840DFF880
:107660001C5111E000F046FA286AC668301D00F08F
:10767000BBF9E86C401EE864686B401E686300F06C
:1076800052FA304600F009F8686B0028EAD1216808
:107690000229F9D3FFF7D1FFF6E710B5044694F8B5
:1076A000510040B9206B00F019F92046BDE81040A8
:1076B00000F014B910BD0128F7D00228FAD0FFF766
:1076C000D4FEFFF7BFFFFEE70D49C86A006810B996
:1076D0004FF0FF3203E0C86AC268D0684268CA66E9
:1076E0007047201D00F080B90122E06A696D824078
:1076F00011436965704700F016FA284670BD000016
:10770000E02300207C2400203046BDE8F2831C4AA0
:107710004FF08051116070470000F8B5174D2F6D84
:107720000C46A96A0646081D00F05EF930B9A86A41
:10773000696DC06A012282409143696516F1010FAB
:1077400005D124B1A86A011D05F138001AE0A86A24
:10775000F6194660BE42A86A05D2011D286BBDE835
:10776000F44000F028B9011DE86A00F024F9E86E41
:10777000864238BFEE66F1BD7C240020E023002065
:1077800004ED00E0BDE8F44000F008B949444C4580
:107790000000000001484068704700BFB0000020B2
:1077A0004018491C1CBFB1F1010100F8012DF9D1AD
:1077B0007047704770477047704770477047704711
:1077C000704700000022FFF7EBBF00002DE9F843EF
:1077D0000446FFF74EFE684FB8684FF000090025D9
:1077E00000BB07F1200307F1200113F0070F40F65B
:1077F000B8300A4604D0CA1DD208D200831AC8186D
:1078000080180838C008C0003A607D60B8604560E4
:107810000560831A5360106050683861F8604FF05B
:107820000040F8614FF05008F869044246D1002C3E
:1078300044D0083414F0070F04D004F1080104F018
:1078400007000C1A002C39D0F868A04236D33E68E5
:10785000394601E0314606467068A04202D23068DF
:107860000028F7D1B868864228D00A6830680860D6
:1078700002F108097268121B112A0CD3311911F098
:10788000070002D000F023F8FEE7301D02517460BB
:10789000084600F04DF87168F8683C69401AF860D5
:1078A000FA68A24288BF2246F8693A6101437160D2
:1078B000356009F007057869401C7861FFF7DFFD46
:1078C00015B100F004F8FEE74846BDE8F28388F3FE
:1078D0001188BFF34F8FBFF36F8F7047002800D11F
:1078E000704738B5A0F10805234C6968E269502358
:1078F000114204D183F31188FFF7EBFFFEE72868FC
:1079000020B183F31188FFF7E4FFFEE7914369603C
:10791000FFF7AFFDE16868684118E160284600F0B4
:1079200007F8A069401CA061BDE83140FFF7A7BD82
:1079300030B511490A4600E01A4613688342FBD36A
:107940005368D418844203D14068C318536010466A
:1079500043681468C518A54208D189688C4204D0D0
:107960006168CB184360246800E00C4604608242E2
:1079700018BF106030BD0000C41100204FF0FF326E
:1079800000F1080182604160C16000F108020261FB
:1079900000210160704700210161704710B5426805
:1079A0004A6093688B6094686160916008610168C7
:1079B000491C016010BD30B50A6812F1010F08BF03
:1079C000036907D000F1080300E023465C682568DE
:1079D000AA42FAD25A684A6091608B605960086185
:1079E0000168491C016030BD4368016982689A6082
:1079F000836842685A604A68824204BF83684B6069
:107A0000002202610868401E086008687047000094
:107A1000490810B54900A0F120034FF08074996126
:107A20001A60DC616FF002020FF20D01596140F83B
:107A3000242D203810BD00004D494A68502012F115
:107A4000010F80F31188BFF34F8FBFF36F8F00D00A
:107A5000FEE7FEE77CB5474A474B10685021984245
:107A600002D100F093F8FEE71068444B984202D12F
:107A700000F08CF8FEE7424B1C780194FF251D7046
:107A80001E783B4C8DF800609DF8000000F050001F
:107A90002070072005E09DF800506D00401E8DF815
:107AA00000509DF800502E06F5D4454215F1030F05
:107AB00003D0A06000F06AF8FEE7000200F4E06086
:107AC000A06001981870116A41F470011162106A87
:107AD00040F07040106200F061F80020606000F03B
:107AE000BBF82848016841F04041016000F0A4F86B
:107AF000002076BD502080F31188BFF34F8FBFF375
:107B00006F8F1B494A68521C012A4A600AD11E49DC
:107B10000A68130606D080F31188BFF34F8FBFF3B6
:107B20006F8FFEE770471249486838B9502080F3DC
:107B30001188BFF34F8FBFF36F8FFEE7401E486081
:107B400008BF80F31188704780B5502080F31188FA
:107B5000BFF34F8FBFF36F8FFFF7E6FC18B10A49F1
:107B60004FF080500860002282F3118801BD0000B0
:107B70007C00002000ED00E071C20F4170C20F4197
:107B800000E400E034EF00E004ED00E081F3118850
:107B9000BFF34F8FBFF36F8F704700000748084B4C
:107BA000002101600022826028221968B1FBF2F2F4
:107BB000521E426007210160704700BF10E000E0E4
:107BC000BC000020EFF30980BFF36F8F264B1A68CB
:107BD0001EF0100F08BF20ED108A20E9F04F106052
:107BE00009B44FF0500080F31188BFF34F8FBFF3FB
:107BF0006F8FFFF7F9FC4FF0000080F3118809BC8C
:107C000019680868B0E8F04F1EF0100F08BFB0EC1C
:107C1000108A80F30988BFF36F8F7047124B196881
:107C20000868B0E8F04F80F30988BFF36F8F4FF01A
:107C3000000080F3118870470C480068006880F3EA
:107C400008884FF0000080F3148862B661B6BFF375
:107C50004F8FBFF36F8F00DFDFF81400016841F42E
:107C600070010160704700000824002008ED00E06A
:107C700088ED00E080B52DED068BB0EE409AF0EE79
:107C8000418AF6EE009A39EE280AB0EE608A20EEBC
:107C9000290A80EE080A00F0CFFBB0EE40AA00F0FF
:107CA000E3FC79EE680A60EEA90AC0EE880A80EE6D
:107CB000800A00F0DBFC80EE0A0ABDEC068BB1EE18
:107CC000400A01BD2DE9F0412DED028B82B08046C6
:107CD00001AB6A4600F0EEFCDFF8F8760198BDF8DB
:107CE0000010786139802D23BDF90000C0EB00122F
:107CF000642110FB03F3002592FBF1FE502210FBE0
:107D000002F093FBF1F6019B90FBF1FC1FFA8EFE53
:107D1000B6B21FFA8CFC462B28BFA3F146052B46B2
:107D2000012204E0B442A8BFA44543DA5B1C0198D9
:107D300083425CD208EB4300011FB1F90240B1F964
:107D40000050A542F2DAB0F90050A542A4BFB0F944
:107D50000240A542EADBB0F90450A542E6DA07F199
:107D6000140444F82230058827F81250521CB0F948
:107D700000407445A8BFA642D4DBB0F90200B1F9B7
:107D8000021000EE103A00EE900AB8EE408AB8EE0B
:107D9000E01A00EE904A00EE101AF8EEE00AB8EE93
:107DA000C00AFFF767FF38EE000A02B0BDEC028B95
:107DB000BDE8F08100EE103AB0F90200B1F902100E
:107DC000B8EE408A00EE100AB8EEC01A00EE104A73
:107DD000F8EEC00A01EE901AB8EEE10AFFF74AFF8A
:107DE00038EE000AFAEE090A30EE200ADDE70FF25B
:107DF0002C60FBF760FD9FED820AD6E738B504469C
:107E0000DFF8D45500224FF4E07100F02AF8002288
:107E10004FF4604100F025F8641E032C20D8DFE801
:107E200004F002060F1701224FF4005113E0012263
:107E30004FF4807100F015F801224FF480410AE000
:107E40000122802100F00DF801224FF4C04102E030
:107E500001224FF4C0712846BDE83840FBF72EB828
:107E600031BD2846FBF72AB8F8B505460E46FAF7A5
:107E7000C6FCDFF86845DFF868752046F9F7D2FEE2
:107E800021680020486232462946DFF85805FCF791
:107E900053FD3868016A41F2111640F244453142FF
:107EA00004BF016A294200F024F800214162012048
:107EB00080F31088DFF83005F9F728FF386801688B
:107EC00041F001010160416AB1F5827FFBD3016A93
:107ED000314204BF016A294200F00BF82046F9F74D
:107EE0006CFE002080F31088BDE8F2400120FBF713
:107EF00093BF03D10268520852000260704700002D
:107F00002DE9F8432DED028B82B005460C4616464E
:107F10000C9F98460DF102023221304600F006FC1B
:107F20006A463221404600F001FCBDF90210DFF83C
:107F3000BC9449423B46324609B2304600F01EFC32
:107F4000BDF9001049423B46424609B2404600F0A6
:107F500015FC39463046FFF7B5FEF0EE040ADFEDBA
:107F6000298A80EE200AB9EE048A30EE280A30EE23
:107F7000080A89ED000A39464046FFF7A3FEB0EE35
:107F8000041A80EE011A31EE281A31EE080AD9EDF2
:107F9000000A89ED010A70EEC01AC9ED021AB7EEA7
:107FA000001AF7EE001AC1EE200A81EE800A30EEC8
:107FB000800A9FED152A20EE022A12EE100A9FED8C
:107FC000981AE860DFED111AD9ED020A99ED000A5E
:107FD00020EE811AC1EE211AC1EE801A81EE800ACC
:107FE0002CB9B1EE400A10EE100A286002E010EE43
:107FF000100A686002B0BDEC028BBDE8F18300009E
:10800000000000000000824300606A472905B53F78
:108010002DE9F84F2DED068B84B0DFF8D4A30AF6D6
:10802000D4010AF1D40201240AF1C006029101929E
:108030009FED7C9ADFF8BC73DFF8BC5341F2111B53
:108040002868016A11EA0B0F02BF016A40F244423C
:10805000114200F0F9F800224262016841F001018A
:1080600001600120FFF7CAFE00F0F4F80120FBF7E1
:10807000D3FE0220FFF7C2FE00F0DCF800F0D4F8D7
:1080800000215046FFF73CFF0320FFF7B7FE00F04A
:10809000E1F80120FBF7C0FE0420FFF7AFFE00F07F
:1080A000C9F800F0C1F801215046FFF729FFDAEDC9
:1080B000008A9AED018A28EEA80A08EE080A00F064
:1080C00087FB8AED020A18EE900ADAED029AFEF7B3
:1080D0004FFD8046894619EE900AFEF749FDC74AD2
:1080E000C74BF9F781F900F0A9F800F081FB00EE29
:1080F000100A00F0A1F98AED040A2868016A11EA61
:108100000B0F02BF016A40F24442114200F09CF89A
:10811000DFEDAC0A30680AEB8001C1ED1C8A81ED0D
:10812000268AC1ED089A9FEDA81A9AED040A60EE1E
:10813000200A80EE811A81ED121A401C0A28306054
:1081400053D3002030600AF1CC020A210AF17000FA
:1081500000F082FB0AF1D0020A210AF1980000F037
:108160007BFB96ED03AAD6ED04AA2AEE0A0A0AEED4
:10817000AA0A00F02DFBF0EE409A19EE900AFEF7E5
:10818000F7FC41EC180B1AEE100AFEF7F1FC8046E2
:10819000894653EC182B9B489B49F9F725F900F0C9
:1081A0004DF800F025FB00EE100A00F045F9DFED78
:1081B000870A80EE200AF5EE40AA20EE09AAF1EE29
:1081C00010FA48BF39EE4AAA51EC180B21F00041D1
:1081D0008E4A8F4BF9F708F83CBFDFED7D9A9FED93
:1081E0007CAAC6ED019A86ED02AA2620FBF714FEB2
:1081F00074B100249AED030A87ED000A87ED010AA5
:10820000BC609AED020A87ED030A87ED040A7C61DF
:10821000DAED030A9AED020A00F020F810E70000F8
:108220000060EA470000B4434FF480600090029B76
:10823000019A704702984FF4806115E602460B469A
:1082400040464946F9F700BA03D101684908490098
:108250000160704701984FF4806105E6F0B56D4C00
:1082600021682069491C032904BF002101202160E5
:1082700063686269A16994ED081AD4ED0E1A5B1C5B
:10828000142B04BF00230122634EA56863603C23C6
:10829000B7886D1C5F43BD4204BF00250121A56066
:1082A0000125E36DE56023B9B0EE401AF0EE601AE7
:1082B000E56530EE410A70EEE10A30EE010A70EE3B
:1082C000A10A94ED0A2A84ED080AC4ED0E0A9FED76
:1082D000401AA8B1206E20B9B0EE402AC4ED100AB1
:1082E000256670EE421A01EE812AD4ED101A84ED53
:1082F000092A70EEE12A42EE811A0020C4ED0F1A1D
:1083000084ED0A2AD4ED0C1A94ED122ABAB1626EE9
:10831000D4ED0F2A94ED093A22B9F0EE431AB0EEEB
:10832000622A656633EE613A72EEC22A43EE011AA2
:1083300002EE812A0022C4ED0B1A84ED112AC4ED4D
:108340000C1A84ED122AA9B394ED111AD4ED141A63
:108350000021F4EE411AF1EE10FA48BF84ED141A30
:10836000D4ED161AB4EE611AF1EE10FA48BF84ED9E
:10837000161AD4ED0B1A94ED132AB4EE612AF1EE1D
:1083800010FA48BFC4ED131A94ED152AF4EE421A00
:10839000F1EE10FA48BFC4ED151A164BA56D1D601D
:1083A00083ED011A256D9D60666DDE60C3ED041AD4
:1083B000E56C5D61A1616261C4ED0D0A84ED070A9F
:1083C0002061F0BD00003443DB0F4940DB0FC940A2
:1083D00000000000802B002000080048082A002030
:1083E000542A002030270020A02A00201C2C002026
:1083F000F0000020F02B0020EC2A00202D431CEB85
:10840000E2361A3F3A8C30E28E79453E9A99999934
:108410009999B93F9827002070000020626164207C
:1084200077617665206F66206563686F2073696782
:108430006E616C200D0A000010EE101A04204FF03F
:108440007E5201EE902A490088BF0820490800EEBC
:10845000101A914214D871EEC00A0F4A31EE801AF8
:10846000914261EE200AF1EEE00A05D980F00400A5
:1084700080EE800A00F0ACBA80EE200A00F0A8BAC4
:10848000490011F1807F9CBF6FF0004100EE101A8F
:10849000AFF3008070470000F404353FDFED620A5F
:1084A00060EE200A10EE902A22F0004101EE101A30
:1084B000DFED5E1AB4EE611AF1EE10FA25D54FF039
:1084C0007C5102F000420A4301EE102A71EE200AAC
:1084D000FDEEE00A10EE901A00296AD0FAEEC90A01
:1084E0009FED531A00EE810ADFED521A00EEA10A49
:1084F0009FED512A00EE820ADFED502A00EEA20A1B
:108500009FED4F1A00EE810A53E010EE101A4B0057
:108510001B1613F1010F0AD14900081610F1010FC3
:1085200002D1090240F07F809FED460A7047490062
:1085300004D1002877D0B7EE000A70474FF07C5185
:1085400002F000420A4301EE102A71EE200A10EEFA
:10855000902A51000DD0090EC1F196011829A8BF2B
:1085600002F0004203DA0029C4BFCA408A4000EE8C
:10857000902A10EE901A490017D09FED331A20EE82
:10858000811ADFED2B1A01EE210A9FED2A2A01EE56
:10859000020ADFED292A01EE220A9FED283A01EEB8
:1085A000030ADFED271A01EE210AFDEEE00A10EEC4
:1085B000901A01F00301081810EE101A21F0004182
:1085C00000EE901A9FED211AF4EE410AF1EE10FA36
:1085D00004D5C10723D5B7EE000A20E0C10760EE3D
:1085E000000A0ED59FED1A0A9FED1A1A00EE801AA6
:1085F000DFED191A41EE201AB7EE000A01EEA00ACB
:108600000DE09FED162ADFED161A40EE821ADFED1F
:10861000152A20EE201A41EEA02A01EE220A800738
:1086200048BFB1EE400A704783F9223F0000004F77
:108630000000C9C600A0FDC00020A2BA000034B3EB
:108640000030C2AEFFFFFF7F00008038000080399D
:108650009349B2BA36A02A3DDFFFFFBE6E8C4CB9FB
:108660004283083CA1AA2ABE002017E710EE101A88
:10867000C1F3C752DAB1992A0FDAC80F21F00041CD
:1086800000EE101AB1F17E5F40F3A281F7EE000A0E
:1086900080EE800A001D00F09BB9FF2A01D14A023A
:1086A00005D1034AC90F42EAC17100EE101A7047A2
:1086B000DB0FC93FF0B50D4604466F1E002034F9AC
:1086C000026BB90884461FD0B4F900E07645BCBF00
:1086D00076460CF10100B4F902E07645BCBF76465F
:1086E0000CF10200B4F904E07645BCBF76460CF10B
:1086F0000300B4F906E008340CF1040C7645BCBF65
:1087000076466046491EDFD117F0030C0BD0614658
:1087100034F9027BBE42BCBF3E46A5EB0C00491EAD
:10872000ACF1010CF4D116801860F0BD70B40346B2
:108730000024880881B012D01E68009635462E04A9
:1087400004EB26445E68009604EB25443546083366
:108750002E0404EB2644401E04EB2544ECD111F01A
:10876000030004D033F9025B6419401EFAD194FB74
:10877000F1F0108001B070BC70470000F0B4044606
:10878000980881B0C1EA014511D0276800973E469C
:1087900096FA15F600961660676800973E4696FAB8
:1087A00015F60096566008340832401EEDD113F0DD
:1087B000030F09D003F0030334F9020B90FA11F010
:1087C0005B1E22F8020BF7D101B0F0BC704700002D
:1087D000B5EEC00AF1EE10FA02D4B1EEC00A70474D
:1087E0006FF0004C00EE10CAAFF30080704700003D
:1087F00001F000428B1AA3F16051B1F5801F0ADB32
:10880000B1F17F6F1FD242EAC102C10071F1004194
:1088100042EB507070470B15C3F10903212B10D2A6
:10882000890241EA905180020128494141F000410A
:1088300021FA03F0C3F12003994071F10041504146
:108840007047100070476FF0000013EB103F5CBFE3
:10885000000E42EAC05070478446880881B09FED00
:108860005B0A00F09E8010F0030313D0DCED000AD9
:108870009CED011A30EE200A30EE010ADCED020A0E
:108880009CED031A30EE200A5B1E30EE010A0CF15B
:10889000100CEBD15FEA900000F08380DCF8003030
:1088A0000093401EDCF80430DDED000A009330EE4A
:1088B000200ADCF80830DDED000A009330EE200AD3
:1088C000DCF80C30DDED000A009330EE200A0CF1EC
:1088D0001003DDED000AD3F800C0CDF800C030EE83
:1088E000200AD3F804C0DDED000ACDF800C030EE58
:1088F000200AD3F808C0DDED000ACDF800C030EE44
:10890000200AD3F80CC0DDED000ACDF800C030EE2F
:10891000200A53F810CFDDED000ACDF800C030EE8C
:10892000200AD3F804C0DDED000ACDF800C030EE17
:10893000200AD3F808C0DDED000ACDF800C030EE03
:10894000200AD3F80CC0DDED000ACDF800C030EEEF
:10895000200A53F810CFDDED000ACDF800C030EE4C
:10896000200AD3F804C0DDED000ACDF800C030EED7
:10897000200AD3F808C0DDED000ACDF800C030EEC3
:10898000200AD3F80CC0DDED000ACDF800C030EEAF
:10899000200ADDED000A30EE200A03F1100C7FF40E
:1089A0007DAF11F0030007D0DCED000A401E30EE71
:1089B000200A0CF1040CF7D100EE901AF8EE600AD0
:1089C00080EE200A82ED000A01B07047000000002E
:1089D0001AA210EE101A43F2A40CC3F6896CF2EC42
:1089E000060A614509DB00EE803A70EE800A83EEEC
:1089F000200A40F0020010EE101A4900D1F1E641C1
:108A00000BD860EE000A20EE203A03EE010A01EED8
:108A1000A02A42EE202A80EE220A400810F0020F1F
:108A200018BFB1EE400A02EB8002D2ED000A30EE30
:108A3000200A28BFB1EE400A70470000D7B3DD3FDF
:108A40006AD5033F2B94A93DB82A593F0000803FC7
:108A5000000080BF00000000920A063FDB0FC93F04
:108A6000920A863FDB0FC93F920A0640DB0F49405E
:108A7000368D2740000000000000000000000000CC
:108A800000000000000000000000000000000000E6
:108A900000000000000000000000000000000000D6
:108AA00000000000000000000000000000000000C6
:108AB00000000000000000000000000000000000B6
:108AC00000000000000000000000000000000000A6
:108AD0000000000000000000000000000000000096
:108AE0000000000000000000000000000000000086
:108AF0000000000000000000000000000000000076
:108B00000000000000000000000000000000000065
:108B10000000000000000000000000000000000055
:108B20000000000000000000000000000000000045
:108B30000000000000000000000000000000000035
:108B40000000000000000000000000000000000025
:108B50000000000000000000000000000000000015
:108B6000000000005B4552524F525D205B25733A76
:108B700025645D20417373657274696F6E2028727D
:108B80006574203D3D2048414C5F4F4B2920666174
:108B9000696C656421207368743330B2C9D1F9CA35
:108BA000A7B0DC0A0D0A00005B4552524F525D200F
:108BB0005B25733A25645D20417373657274696F38
:108BC0006E202828746D705F74656D646174612E09
:108BD0006656616C7565203E3D202D343029202677
:108BE000262028746D705F74656D646174612E66F3
:108BF00056616C7565203C3D203835292920666119
:108C0000696C656421207368743330CEC2B6C8D6EF
:108C1000B5D0A3D1E9CAA7B0DC0A0D0A0000000054
:108C20005B4552524F525D205B25733A25645D20AF
:108C3000417373657274696F6E202828746D705F5C
:108C400068756D69646174612E6656616C75652026
:108C50003E3D2030292026262028746D705F6875DF
:108C60006D69646174612E6656616C7565203C3D6A
:108C7000203130302929206661696C6564212073B8
:108C800068743330CAAAB6C8D6B5D0A3D1E9CAA78A
:108C9000B0DC0A0D0A000000453A5C595C494152BB
:108CA0005C6D6963726F5F636C696D6174655C4173
:108CB00070705C5372635C6672745F70726F746F15
:108CC000636F6C2E630000005B4552524F525D2073
:108CD0005B25733A25645D20417373657274696F17
:108CE0006E202873746172745F7265675F6164647B
:108CF00072203C2031303029206661696C65642126
:108D000020E8AFBBE58F96E5AF84E5AD98E599A87F
:108D1000E8B5B7E5A78BE59CB0E59D80E99499E8B7
:108D2000AFAF25640A0D0A005B4552524F525D20D9
:108D30005B25733A25645D20417373657274696FB6
:108D40006E20287265675F6E756D203C2031303073
:108D500029206661696C65642120E8AFBBE58F96C8
:108D6000E5AF84E5AD98E599A8E695B0E9878FE988
:108D70009499E8AFAF25640A0D0A00005B45525292
:108D80004F525D205B25733A25645D204173736506
:108D90007274696F6E20286765745F74656D705FAB
:108DA00068756D695F646174612826675F73744DCF
:108DB00063735F506172612E74656D70657261746A
:108DC0007572652C2026675F73744D63735F506105
:108DD00072612E68756D69646974792929206661EC
:108DE000696C65642120E98787E99B867368743321
:108DF00030E6B8A9E6B9BFE5BAA6E695B0E68DAE0D
:108E0000E5A4B1E8B4A50A0D0A000000FEE7FEE7FC
:108E1000FEE7FEE7FEE770472548FCF75BBC80B540
:108E20002448F9F73BF8BDE802402348F9F736B883
:108E300038B5224D224C2846FCF7D2FD01222146AE
:108E40002846FCF797FD1F4800684169C268491C25
:108E500091FBF2F302FB13110269914205D02178D4
:108E6000BDE834400830FDF717BE31BD70B5164E71
:108E7000164D3046FCF7B4FD15490C680122294611
:108E80003046FCF777FD6069E168401C90FBF1F229
:108E900001FB12002169884206D0297804F10800FC
:108EA000BDE87040FDF7F8BD70BD0A48FCF798BDFD
:108EB000382B002070290020EC2A002008250020F3
:108EC00090250020F01F0020942500201C26002063
:108ED0002021002020260020453A5C595C4941525F
:108EE0005C6D6963726F5F636C696D6174655C442E
:108EF0007269766572735C53687433785C736874F6
:108F000033302E63000000005B4552524F525D200B
:108F10005B25733A25645D20417373657274696FD4
:108F20006E20286765745F74656D705F68756D6924
:108F30005F64617461282674656D702C20266875E5
:108F40006D692929206661696C65642120212121D0
:108F500053656E736F7220536874333020436865B5
:108F6000636B204661696C65640A0D0A00000000AD
:108F700053656E736F722053687433302043686595
:108F8000636B204F4B2E0D0A2054656D703A252ED1
:108F900032662C48756D693A252E32660D0A00003E
:108FA0000E48016841F47001016000220C49086814
:108FB00040F0010008608A604FF480520B68094855
:108FC00003400B60CA6000200B68074A23F480232B
:108FD0000B6088614FF000611160704788ED00E020
:108FE00000100240FFFFF6EA08ED00E0000000007C
:108FF00000000000010203040607080930B4002540
:1090000012E050F8042BD30744BF4A44521E091FF4
:10901000042942F8045BFAD213468C0744BF15803A
:109020009B1CC90748BF1D7050F8041B0029E8D1DC
:1090300030BC7047A0860100400D0300801A060076
:1090400000350C0040420F0080841E0000093D00E6
:1090500000127A000024F40000366E010048E80196
:10906000006CDC0210B5074979441831064C7C4489
:10907000163404E00A68081D114488470146A142DD
:10908000F8D110BD2C000000480000004EF68851B9
:10909000CEF20001086840F470000860BFF34F8F03
:1090A000BFF36F8F4FF00170E1EE100A70470000C0
:1090B0004DFFFFFF442B0000F000002000000000E7
:1090C0009B7FFFFFE0010000460100000000002040
:1090D00000F00DF8002801D0FFF7C4FFAFF30080C7
:1090E0000020AFF30080F9F7BFFC00F002F8012088
:1090F000704700F001B8000007463846F8F746FD13
:10910000FBE700000548014603B4684680F3098880
:10911000AFF30080FFF7BAFFFFF7DAFFA5EDF5FE2A
:109120000148804701480047A18F000805910008C9
:1091300064656661756C745461736B00616E656D16
:109140006F6D657465720000000000000102030489
:10915000FFF7FEBFFFF7FEBFFFF7FEBFFFF7FEBF43
:10916000FFF7FEBFFFF7FEBFFFF7FEBFFFF7FEBF33
:10917000FFF7FEBFFFF7FEBFFFF7FEBFFFF7FEBF23
:10918000FFF7FEBFFFF7FEBFFFF7FEBFFFF7FEBF13
:10919000FFF7FEBFFFF7FEBFFFF7FEBFFFF7FEBF03
:1091A000FFF7FEBFFFF7FEBFFFF7FEBFFFF7FEBFF3
:1091B000FFF7FEBFFFF7FEBFFFF7FEBFFFF7FEBFE3
:1091C000FFF7FEBFFFF7FEBFFFF7FEBFFFF7FEBFD3
:1091D000FFF7FEBFFFF7FEBFFFF7FEBFFFF7FEBFC3
:1091E000FFF7FEBFFFF7FEBFFFF7FEBFFFF7FEBFB3
:1091F000FFF7FEBFFFF7FEBFFFF7FEBFFFF7FEBFA3
:10920000FFF7FEBFFFF7FEBFFFF7FEBFFFF7FEBF92
:10921000FFF7FEBFFFF7FEBFFFF7FEBFFFF7FEBF82
:10922000FFF7FEBFFFF7FEBFFFF7FEBFFFF7FEBF72
:10923000FFF7FEBFFFF7FEBFFFF7FEBFFFF7FEBF62
:10924000FFF7FEBFFFF7FEBFFFF7FEBFFFF7FEBF52
:10925000FFF7FEBFFFF7FEBFFFF7FEBFFFF7FEBF42
:10926000FFF7FEBFFFF7FEBFFFF7FEBFFFF7FEBF32
:10927000FFF7FEBFFFF7FEBFFFF7FEBFFFF7FEBF22
:10928000FFF7FEBFFFF7FEBFFFF7FEBFFFF7FEBF12
:10929000FFF7FEBFFFF7FEBFFFF7FEBFFFF7FEBF02
:1092A000FFF7FEBF0003FD0004716D000810FD0014
:1092B000032D6E0008FC00047B6C000801FD000417
:1092C000836C000802FD0004A96C000803FD000483
:1092D000B16C000804FD0004B96C000805FD000431
:1092E000C16C000806FD0004C96C000807FD0004FD
:1092F000D16C000808FD0004D96C000809FD0004C9
:10930000DF6C00080AFD0004E56C000814FD00088D
:10931000EB6C0008553080250AFD000016F900FCB2
:10932000AADC00088800062C062C000001F90000C9
:1093300010FC0008093D00000100008025ED00043C
:079340000300008025EE0090
:040000050800910559
:00000001FF
